

Microchip Technology PIC LITE Macro Assembler V1.12 build 49521 
                                                                                               Sat Dec 29 09:51:30 2012

HI-TECH Software Omniscient Code Generator (Lite mode) build 49521
     1  0000                     opt subtitle "HI-TECH Software Omniscient Code Generator (Lite mode) build 49521"
     2                           opt subtitle "HI-TECH Software Omniscient Code Generator (Lite mode) build 49521"
     3                           
     4                           opt pagewidth 120
     5                           
     6                           	opt lm
     7                           
     8                           	processor	16F1827
     9                           clrc	macro
    10  0000                     	endm
    11                           opt subtitle "HI-TECH Software Omniscient Code Generator (Lite mode) build 49521"
    12                           
    13  0000                     	endm
    14                           opt subtitle "HI-TECH Software Omniscient Code Generator (Lite mode) build 49521"
    15                           
    16  0000                     	endm
    17                           opt subtitle "HI-TECH Software Omniscient Code Generator (Lite mode) build 49521"
    18                           
    19  0000                     	endm
    20                           opt subtitle "HI-TECH Software Omniscient Code Generator (Lite mode) build 49521"
    21                           
    22  0000                     	endm
    23                           opt subtitle "HI-TECH Software Omniscient Code Generator (Lite mode) build 49521"
    24                           
    25  0000                     	endm
    26                           opt subtitle "HI-TECH Software Omniscient Code Generator (Lite mode) build 49521"
    27                           
    28  0000                     	endm
    29                           opt subtitle "HI-TECH Software Omniscient Code Generator (Lite mode) build 49521"
    30                           
    31  0000                     	endm
    32  0000                     indf	equ	0
    33  0000                     indf0	equ	0
    34  0001                     indf1	equ	1
    35  0002                     pc	equ	2
    36  0002                     pcl	equ	2
    37  0003                     status	equ	3
    38  0004                     fsr0l	equ	4
    39  0005                     fsr0h	equ	5
    40  0006                     fsr1l	equ	6
    41  0007                     fsr1h	equ	7
    42  0008                     bsr	equ	8
    43  0009                     wreg	equ	9
    44  000B                     intcon	equ	11
    45  0001                     c	equ	1
    46  0000                     z	equ	0
    47  000A                     pclath	equ	10
    48                           opt subtitle "HI-TECH Software Omniscient Code Generator (Lite mode) build 49521"
    49  0000                     INDF0 equ 00h ;# 
    50                           opt subtitle "HI-TECH Software Omniscient Code Generator (Lite mode) build 49521"
    51  0001                     INDF1 equ 01h ;# 
    52                           opt subtitle "HI-TECH Software Omniscient Code Generator (Lite mode) build 49521"
    53  0002                     PCL equ 02h ;# 
    54                           opt subtitle "HI-TECH Software Omniscient Code Generator (Lite mode) build 49521"
    55  0003                     STATUS equ 03h ;# 
    56                           opt subtitle "HI-TECH Software Omniscient Code Generator (Lite mode) build 49521"
    57  0004                     FSR0L equ 04h ;# 
    58                           opt subtitle "HI-TECH Software Omniscient Code Generator (Lite mode) build 49521"
    59  0005                     FSR0H equ 05h ;# 
    60                           opt subtitle "HI-TECH Software Omniscient Code Generator (Lite mode) build 49521"
    61  0006                     FSR1L equ 06h ;# 
    62                           opt subtitle "HI-TECH Software Omniscient Code Generator (Lite mode) build 49521"
    63  0007                     FSR1H equ 07h ;# 
    64                           opt subtitle "HI-TECH Software Omniscient Code Generator (Lite mode) build 49521"
    65  0008                     BSR equ 08h ;# 
    66                           opt subtitle "HI-TECH Software Omniscient Code Generator (Lite mode) build 49521"
    67  0009                     WREG equ 09h ;# 
    68                           opt subtitle "HI-TECH Software Omniscient Code Generator (Lite mode) build 49521"
    69  000A                     PCLATH equ 0Ah ;# 
    70                           opt subtitle "HI-TECH Software Omniscient Code Generator (Lite mode) build 49521"
    71  000B                     INTCON equ 0Bh ;# 
    72                           opt subtitle "HI-TECH Software Omniscient Code Generator (Lite mode) build 49521"
    73  000C                     PORTA equ 0Ch ;# 
    74                           opt subtitle "HI-TECH Software Omniscient Code Generator (Lite mode) build 49521"
    75  000D                     PORTB equ 0Dh ;# 
    76                           opt subtitle "HI-TECH Software Omniscient Code Generator (Lite mode) build 49521"
    77  0011                     PIR1 equ 011h ;# 
    78                           opt subtitle "HI-TECH Software Omniscient Code Generator (Lite mode) build 49521"
    79  0012                     PIR2 equ 012h ;# 
    80                           opt subtitle "HI-TECH Software Omniscient Code Generator (Lite mode) build 49521"
    81  0013                     PIR3 equ 013h ;# 
    82                           opt subtitle "HI-TECH Software Omniscient Code Generator (Lite mode) build 49521"
    83  0014                     PIR4 equ 014h ;# 
    84                           opt subtitle "HI-TECH Software Omniscient Code Generator (Lite mode) build 49521"
    85  0015                     TMR0 equ 015h ;# 
    86                           opt subtitle "HI-TECH Software Omniscient Code Generator (Lite mode) build 49521"
    87  0016                     TMR1 equ 016h ;# 
    88                           opt subtitle "HI-TECH Software Omniscient Code Generator (Lite mode) build 49521"
    89  0016                     TMR1L equ 016h ;# 
    90                           opt subtitle "HI-TECH Software Omniscient Code Generator (Lite mode) build 49521"
    91  0017                     TMR1H equ 017h ;# 
    92                           opt subtitle "HI-TECH Software Omniscient Code Generator (Lite mode) build 49521"
    93  0018                     T1CON equ 018h ;# 
    94                           opt subtitle "HI-TECH Software Omniscient Code Generator (Lite mode) build 49521"
    95  0019                     T1GCON equ 019h ;# 
    96                           opt subtitle "HI-TECH Software Omniscient Code Generator (Lite mode) build 49521"
    97  001A                     TMR2 equ 01Ah ;# 
    98                           opt subtitle "HI-TECH Software Omniscient Code Generator (Lite mode) build 49521"
    99  001B                     PR2 equ 01Bh ;# 
   100                           opt subtitle "HI-TECH Software Omniscient Code Generator (Lite mode) build 49521"
   101  001C                     T2CON equ 01Ch ;# 
   102                           opt subtitle "HI-TECH Software Omniscient Code Generator (Lite mode) build 49521"
   103  001E                     CPSCON0 equ 01Eh ;# 
   104                           opt subtitle "HI-TECH Software Omniscient Code Generator (Lite mode) build 49521"
   105  001F                     CPSCON1 equ 01Fh ;# 
   106                           opt subtitle "HI-TECH Software Omniscient Code Generator (Lite mode) build 49521"
   107  008C                     TRISA equ 08Ch ;# 
   108                           opt subtitle "HI-TECH Software Omniscient Code Generator (Lite mode) build 49521"
   109  008D                     TRISB equ 08Dh ;# 
   110                           opt subtitle "HI-TECH Software Omniscient Code Generator (Lite mode) build 49521"
   111  0091                     PIE1 equ 091h ;# 
   112                           opt subtitle "HI-TECH Software Omniscient Code Generator (Lite mode) build 49521"
   113  0092                     PIE2 equ 092h ;# 
   114                           opt subtitle "HI-TECH Software Omniscient Code Generator (Lite mode) build 49521"
   115  0093                     PIE3 equ 093h ;# 
   116                           opt subtitle "HI-TECH Software Omniscient Code Generator (Lite mode) build 49521"
   117  0094                     PIE4 equ 094h ;# 
   118                           opt subtitle "HI-TECH Software Omniscient Code Generator (Lite mode) build 49521"
   119  0095                     OPTION_REG equ 095h ;# 
   120                           opt subtitle "HI-TECH Software Omniscient Code Generator (Lite mode) build 49521"
   121  0096                     PCON equ 096h ;# 
   122                           opt subtitle "HI-TECH Software Omniscient Code Generator (Lite mode) build 49521"
   123  0097                     WDTCON equ 097h ;# 
   124                           opt subtitle "HI-TECH Software Omniscient Code Generator (Lite mode) build 49521"
   125  0098                     OSCTUNE equ 098h ;# 
   126                           opt subtitle "HI-TECH Software Omniscient Code Generator (Lite mode) build 49521"
   127  0099                     OSCCON equ 099h ;# 
   128                           opt subtitle "HI-TECH Software Omniscient Code Generator (Lite mode) build 49521"
   129  009A                     OSCSTAT equ 09Ah ;# 
   130                           opt subtitle "HI-TECH Software Omniscient Code Generator (Lite mode) build 49521"
   131  009B                     ADRES equ 09Bh ;# 
   132                           opt subtitle "HI-TECH Software Omniscient Code Generator (Lite mode) build 49521"
   133  009B                     ADRESL equ 09Bh ;# 
   134                           opt subtitle "HI-TECH Software Omniscient Code Generator (Lite mode) build 49521"
   135  009C                     ADRESH equ 09Ch ;# 
   136                           opt subtitle "HI-TECH Software Omniscient Code Generator (Lite mode) build 49521"
   137  009D                     ADCON0 equ 09Dh ;# 
   138                           opt subtitle "HI-TECH Software Omniscient Code Generator (Lite mode) build 49521"
   139  009E                     ADCON1 equ 09Eh ;# 
   140                           opt subtitle "HI-TECH Software Omniscient Code Generator (Lite mode) build 49521"
   141  010C                     LATA equ 010Ch ;# 
   142                           opt subtitle "HI-TECH Software Omniscient Code Generator (Lite mode) build 49521"
   143  010D                     LATB equ 010Dh ;# 
   144                           opt subtitle "HI-TECH Software Omniscient Code Generator (Lite mode) build 49521"
   145  0111                     CM1CON0 equ 0111h ;# 
   146                           opt subtitle "HI-TECH Software Omniscient Code Generator (Lite mode) build 49521"
   147  0112                     CM1CON1 equ 0112h ;# 
   148                           opt subtitle "HI-TECH Software Omniscient Code Generator (Lite mode) build 49521"
   149  0113                     CM2CON0 equ 0113h ;# 
   150                           opt subtitle "HI-TECH Software Omniscient Code Generator (Lite mode) build 49521"
   151  0114                     CM2CON1 equ 0114h ;# 
   152                           opt subtitle "HI-TECH Software Omniscient Code Generator (Lite mode) build 49521"
   153  0115                     CMOUT equ 0115h ;# 
   154                           opt subtitle "HI-TECH Software Omniscient Code Generator (Lite mode) build 49521"
   155  0116                     BORCON equ 0116h ;# 
   156                           opt subtitle "HI-TECH Software Omniscient Code Generator (Lite mode) build 49521"
   157  0117                     FVRCON equ 0117h ;# 
   158                           opt subtitle "HI-TECH Software Omniscient Code Generator (Lite mode) build 49521"
   159  0118                     DACCON0 equ 0118h ;# 
   160                           opt subtitle "HI-TECH Software Omniscient Code Generator (Lite mode) build 49521"
   161  0119                     DACCON1 equ 0119h ;# 
   162                           opt subtitle "HI-TECH Software Omniscient Code Generator (Lite mode) build 49521"
   163  011A                     SRCON0 equ 011Ah ;# 
   164                           opt subtitle "HI-TECH Software Omniscient Code Generator (Lite mode) build 49521"
   165  011B                     SRCON1 equ 011Bh ;# 
   166                           opt subtitle "HI-TECH Software Omniscient Code Generator (Lite mode) build 49521"
   167  011D                     APFCON0 equ 011Dh ;# 
   168                           opt subtitle "HI-TECH Software Omniscient Code Generator (Lite mode) build 49521"
   169  011E                     APFCON1 equ 011Eh ;# 
   170                           opt subtitle "HI-TECH Software Omniscient Code Generator (Lite mode) build 49521"
   171  018C                     ANSELA equ 018Ch ;# 
   172                           opt subtitle "HI-TECH Software Omniscient Code Generator (Lite mode) build 49521"
   173  018D                     ANSELB equ 018Dh ;# 
   174                           opt subtitle "HI-TECH Software Omniscient Code Generator (Lite mode) build 49521"
   175  0191                     EEADR equ 0191h ;# 
   176                           opt subtitle "HI-TECH Software Omniscient Code Generator (Lite mode) build 49521"
   177  0191                     EEADRL equ 0191h ;# 
   178                           opt subtitle "HI-TECH Software Omniscient Code Generator (Lite mode) build 49521"
   179  0192                     EEADRH equ 0192h ;# 
   180                           opt subtitle "HI-TECH Software Omniscient Code Generator (Lite mode) build 49521"
   181  0193                     EEDAT equ 0193h ;# 
   182                           opt subtitle "HI-TECH Software Omniscient Code Generator (Lite mode) build 49521"
   183  0193                     EEDATL equ 0193h ;# 
   184                           opt subtitle "HI-TECH Software Omniscient Code Generator (Lite mode) build 49521"
   185  0193                     EEDATA equ 0193h ;# 
   186                           opt subtitle "HI-TECH Software Omniscient Code Generator (Lite mode) build 49521"
   187  0194                     EEDATH equ 0194h ;# 
   188                           opt subtitle "HI-TECH Software Omniscient Code Generator (Lite mode) build 49521"
   189  0195                     EECON1 equ 0195h ;# 
   190                           opt subtitle "HI-TECH Software Omniscient Code Generator (Lite mode) build 49521"
   191  0196                     EECON2 equ 0196h ;# 
   192                           opt subtitle "HI-TECH Software Omniscient Code Generator (Lite mode) build 49521"
   193  0199                     RCREG equ 0199h ;# 
   194                           opt subtitle "HI-TECH Software Omniscient Code Generator (Lite mode) build 49521"
   195  019A                     TXREG equ 019Ah ;# 
   196                           opt subtitle "HI-TECH Software Omniscient Code Generator (Lite mode) build 49521"
   197  019B                     SPBRGL equ 019Bh ;# 
   198                           opt subtitle "HI-TECH Software Omniscient Code Generator (Lite mode) build 49521"
   199  019B                     SPBRG equ 019Bh ;# 
   200                           opt subtitle "HI-TECH Software Omniscient Code Generator (Lite mode) build 49521"
   201  019C                     SPBRGH equ 019Ch ;# 
   202                           opt subtitle "HI-TECH Software Omniscient Code Generator (Lite mode) build 49521"
   203  019D                     RCSTA equ 019Dh ;# 
   204                           opt subtitle "HI-TECH Software Omniscient Code Generator (Lite mode) build 49521"
   205  019E                     TXSTA equ 019Eh ;# 
   206                           opt subtitle "HI-TECH Software Omniscient Code Generator (Lite mode) build 49521"
   207  019F                     BAUDCON equ 019Fh ;# 
   208                           opt subtitle "HI-TECH Software Omniscient Code Generator (Lite mode) build 49521"
   209  020C                     WPUA equ 020Ch ;# 
   210                           opt subtitle "HI-TECH Software Omniscient Code Generator (Lite mode) build 49521"
   211  020D                     WPUB equ 020Dh ;# 
   212                           opt subtitle "HI-TECH Software Omniscient Code Generator (Lite mode) build 49521"
   213  0211                     SSP1BUF equ 0211h ;# 
   214                           opt subtitle "HI-TECH Software Omniscient Code Generator (Lite mode) build 49521"
   215  0211                     SSPBUF equ 0211h ;# 
   216                           opt subtitle "HI-TECH Software Omniscient Code Generator (Lite mode) build 49521"
   217  0212                     SSP1ADD equ 0212h ;# 
   218                           opt subtitle "HI-TECH Software Omniscient Code Generator (Lite mode) build 49521"
   219  0212                     SSPADD equ 0212h ;# 
   220                           opt subtitle "HI-TECH Software Omniscient Code Generator (Lite mode) build 49521"
   221  0213                     SSP1MSK equ 0213h ;# 
   222                           opt subtitle "HI-TECH Software Omniscient Code Generator (Lite mode) build 49521"
   223  0213                     SSPMSK equ 0213h ;# 
   224                           opt subtitle "HI-TECH Software Omniscient Code Generator (Lite mode) build 49521"
   225  0214                     SSP1STAT equ 0214h ;# 
   226                           opt subtitle "HI-TECH Software Omniscient Code Generator (Lite mode) build 49521"
   227  0214                     SSPSTAT equ 0214h ;# 
   228                           opt subtitle "HI-TECH Software Omniscient Code Generator (Lite mode) build 49521"
   229  0215                     SSP1CON1 equ 0215h ;# 
   230                           opt subtitle "HI-TECH Software Omniscient Code Generator (Lite mode) build 49521"
   231  0215                     SSPCON1 equ 0215h ;# 
   232                           opt subtitle "HI-TECH Software Omniscient Code Generator (Lite mode) build 49521"
   233  0215                     SSPCON equ 0215h ;# 
   234                           opt subtitle "HI-TECH Software Omniscient Code Generator (Lite mode) build 49521"
   235  0216                     SSP1CON2 equ 0216h ;# 
   236                           opt subtitle "HI-TECH Software Omniscient Code Generator (Lite mode) build 49521"
   237  0216                     SSPCON2 equ 0216h ;# 
   238                           opt subtitle "HI-TECH Software Omniscient Code Generator (Lite mode) build 49521"
   239  0217                     SSP1CON3 equ 0217h ;# 
   240                           opt subtitle "HI-TECH Software Omniscient Code Generator (Lite mode) build 49521"
   241  0217                     SSPCON3 equ 0217h ;# 
   242                           opt subtitle "HI-TECH Software Omniscient Code Generator (Lite mode) build 49521"
   243  0219                     SSP2BUF equ 0219h ;# 
   244                           opt subtitle "HI-TECH Software Omniscient Code Generator (Lite mode) build 49521"
   245  021A                     SSP2ADD equ 021Ah ;# 
   246                           opt subtitle "HI-TECH Software Omniscient Code Generator (Lite mode) build 49521"
   247  021B                     SSP2MSK equ 021Bh ;# 
   248                           opt subtitle "HI-TECH Software Omniscient Code Generator (Lite mode) build 49521"
   249  021C                     SSP2STAT equ 021Ch ;# 
   250                           opt subtitle "HI-TECH Software Omniscient Code Generator (Lite mode) build 49521"
   251  021D                     SSP2CON1 equ 021Dh ;# 
   252                           opt subtitle "HI-TECH Software Omniscient Code Generator (Lite mode) build 49521"
   253  021E                     SSP2CON2 equ 021Eh ;# 
   254                           opt subtitle "HI-TECH Software Omniscient Code Generator (Lite mode) build 49521"
   255  021F                     SSP2CON3 equ 021Fh ;# 
   256                           opt subtitle "HI-TECH Software Omniscient Code Generator (Lite mode) build 49521"
   257  0291                     CCPR1L equ 0291h ;# 
   258                           opt subtitle "HI-TECH Software Omniscient Code Generator (Lite mode) build 49521"
   259  0292                     CCPR1H equ 0292h ;# 
   260                           opt subtitle "HI-TECH Software Omniscient Code Generator (Lite mode) build 49521"
   261  0293                     CCP1CON equ 0293h ;# 
   262                           opt subtitle "HI-TECH Software Omniscient Code Generator (Lite mode) build 49521"
   263  0294                     PWM1CON equ 0294h ;# 
   264                           opt subtitle "HI-TECH Software Omniscient Code Generator (Lite mode) build 49521"
   265  0295                     CCP1AS equ 0295h ;# 
   266                           opt subtitle "HI-TECH Software Omniscient Code Generator (Lite mode) build 49521"
   267  0295                     ECCP1AS equ 0295h ;# 
   268                           opt subtitle "HI-TECH Software Omniscient Code Generator (Lite mode) build 49521"
   269  0296                     PSTR1CON equ 0296h ;# 
   270                           opt subtitle "HI-TECH Software Omniscient Code Generator (Lite mode) build 49521"
   271  0298                     CCPR2L equ 0298h ;# 
   272                           opt subtitle "HI-TECH Software Omniscient Code Generator (Lite mode) build 49521"
   273  0299                     CCPR2H equ 0299h ;# 
   274                           opt subtitle "HI-TECH Software Omniscient Code Generator (Lite mode) build 49521"
   275  029A                     CCP2CON equ 029Ah ;# 
   276                           opt subtitle "HI-TECH Software Omniscient Code Generator (Lite mode) build 49521"
   277  029B                     PWM2CON equ 029Bh ;# 
   278                           opt subtitle "HI-TECH Software Omniscient Code Generator (Lite mode) build 49521"
   279  029C                     CCP2AS equ 029Ch ;# 
   280                           opt subtitle "HI-TECH Software Omniscient Code Generator (Lite mode) build 49521"
   281  029C                     ECCP2AS equ 029Ch ;# 
   282                           opt subtitle "HI-TECH Software Omniscient Code Generator (Lite mode) build 49521"
   283  029D                     PSTR2CON equ 029Dh ;# 
   284                           opt subtitle "HI-TECH Software Omniscient Code Generator (Lite mode) build 49521"
   285  029E                     CCPTMRS equ 029Eh ;# 
   286                           opt subtitle "HI-TECH Software Omniscient Code Generator (Lite mode) build 49521"
   287  029E                     CCPTMRS0 equ 029Eh ;# 
   288                           opt subtitle "HI-TECH Software Omniscient Code Generator (Lite mode) build 49521"
   289  0311                     CCPR3L equ 0311h ;# 
   290                           opt subtitle "HI-TECH Software Omniscient Code Generator (Lite mode) build 49521"
   291  0312                     CCPR3H equ 0312h ;# 
   292                           opt subtitle "HI-TECH Software Omniscient Code Generator (Lite mode) build 49521"
   293  0313                     CCP3CON equ 0313h ;# 
   294                           opt subtitle "HI-TECH Software Omniscient Code Generator (Lite mode) build 49521"
   295  0318                     CCPR4L equ 0318h ;# 
   296                           opt subtitle "HI-TECH Software Omniscient Code Generator (Lite mode) build 49521"
   297  0319                     CCPR4H equ 0319h ;# 
   298                           opt subtitle "HI-TECH Software Omniscient Code Generator (Lite mode) build 49521"
   299  031A                     CCP4CON equ 031Ah ;# 
   300                           opt subtitle "HI-TECH Software Omniscient Code Generator (Lite mode) build 49521"
   301  0394                     IOCBP equ 0394h ;# 
   302                           opt subtitle "HI-TECH Software Omniscient Code Generator (Lite mode) build 49521"
   303  0395                     IOCBN equ 0395h ;# 
   304                           opt subtitle "HI-TECH Software Omniscient Code Generator (Lite mode) build 49521"
   305  0396                     IOCBF equ 0396h ;# 
   306                           opt subtitle "HI-TECH Software Omniscient Code Generator (Lite mode) build 49521"
   307  039A                     CLKRCON equ 039Ah ;# 
   308                           opt subtitle "HI-TECH Software Omniscient Code Generator (Lite mode) build 49521"
   309  039C                     MDCON equ 039Ch ;# 
   310                           opt subtitle "HI-TECH Software Omniscient Code Generator (Lite mode) build 49521"
   311  039D                     MDSRC equ 039Dh ;# 
   312                           opt subtitle "HI-TECH Software Omniscient Code Generator (Lite mode) build 49521"
   313  039E                     MDCARL equ 039Eh ;# 
   314                           opt subtitle "HI-TECH Software Omniscient Code Generator (Lite mode) build 49521"
   315  039F                     MDCARH equ 039Fh ;# 
   316                           opt subtitle "HI-TECH Software Omniscient Code Generator (Lite mode) build 49521"
   317  0415                     TMR4 equ 0415h ;# 
   318                           opt subtitle "HI-TECH Software Omniscient Code Generator (Lite mode) build 49521"
   319  0416                     PR4 equ 0416h ;# 
   320                           opt subtitle "HI-TECH Software Omniscient Code Generator (Lite mode) build 49521"
   321  0417                     T4CON equ 0417h ;# 
   322                           opt subtitle "HI-TECH Software Omniscient Code Generator (Lite mode) build 49521"
   323  041C                     TMR6 equ 041Ch ;# 
   324                           opt subtitle "HI-TECH Software Omniscient Code Generator (Lite mode) build 49521"
   325  041D                     PR6 equ 041Dh ;# 
   326                           opt subtitle "HI-TECH Software Omniscient Code Generator (Lite mode) build 49521"
   327  041E                     T6CON equ 041Eh ;# 
   328                           opt subtitle "HI-TECH Software Omniscient Code Generator (Lite mode) build 49521"
   329  0FE4                     STATUS_SHAD equ 0FE4h ;# 
   330                           opt subtitle "HI-TECH Software Omniscient Code Generator (Lite mode) build 49521"
   331  0FE5                     WREG_SHAD equ 0FE5h ;# 
   332                           opt subtitle "HI-TECH Software Omniscient Code Generator (Lite mode) build 49521"
   333  0FE6                     BSR_SHAD equ 0FE6h ;# 
   334                           opt subtitle "HI-TECH Software Omniscient Code Generator (Lite mode) build 49521"
   335  0FE7                     PCLATH_SHAD equ 0FE7h ;# 
   336                           opt subtitle "HI-TECH Software Omniscient Code Generator (Lite mode) build 49521"
   337  0FE8                     FSR0L_SHAD equ 0FE8h ;# 
   338                           opt subtitle "HI-TECH Software Omniscient Code Generator (Lite mode) build 49521"
   339  0FE9                     FSR0H_SHAD equ 0FE9h ;# 
   340                           opt subtitle "HI-TECH Software Omniscient Code Generator (Lite mode) build 49521"
   341  0FEA                     FSR1L_SHAD equ 0FEAh ;# 
   342                           opt subtitle "HI-TECH Software Omniscient Code Generator (Lite mode) build 49521"
   343  0FEB                     FSR1H_SHAD equ 0FEBh ;# 
   344                           opt subtitle "HI-TECH Software Omniscient Code Generator (Lite mode) build 49521"
   345  0FED                     STKPTR equ 0FEDh ;# 
   346                           opt subtitle "HI-TECH Software Omniscient Code Generator (Lite mode) build 49521"
   347  0FEE                     TOSL equ 0FEEh ;# 
   348                           opt subtitle "HI-TECH Software Omniscient Code Generator (Lite mode) build 49521"
   349  0FEF                     TOSH equ 0FEFh ;# 
   350                           opt subtitle "HI-TECH Software Omniscient Code Generator (Lite mode) build 49521"
   351                           
   352                           opt pagewidth 120
   353                           
   354                           	opt lm
   355                           
   356                           	processor	16F1827
   357                           clrc	macro
   358                           	bcf	3,0
   359                           	endm
   360                           clrz	macro
   361                           	bcf	3,2
   362                           	endm
   363  01CF                     __pidataBANK0:
   364                           opt subtitle "HI-TECH Software Omniscient Code Generator (Lite mode) build 49521"
   365                           
   366                           opt pagewidth 120
   367                           
   368  01CF  340D               	retlw	0Dh
   369  01D0  340A               	retlw	0Ah
   370  01D1  342A               	retlw	02Ah
   371  01D2  342A               	retlw	02Ah
   372  01D3  342A               	retlw	02Ah
   373  01D4  345F               	retlw	05Fh
   374  01D5  345F               	retlw	05Fh
   375  01D6  3453               	retlw	053h
   376  01D7  3477               	retlw	077h
   377  01D8  3469               	retlw	069h
   378  01D9  3474               	retlw	074h
   379  01DA  3463               	retlw	063h
   380  01DB  3468               	retlw	068h
   381  01DC  3432               	retlw	032h
   382  01DD  345F               	retlw	05Fh
   383  01DE  345F               	retlw	05Fh
   384  01DF  3450               	retlw	050h
   385  01E0  3472               	retlw	072h
   386  01E1  3465               	retlw	065h
   387  01E2  3473               	retlw	073h
   388  01E3  3473               	retlw	073h
   389  01E4  3465               	retlw	065h
   390  01E5  3464               	retlw	064h
   391  01E6  345F               	retlw	05Fh
   392  01E7  345F               	retlw	05Fh
   393  01E8  342A               	retlw	02Ah
   394  01E9  342A               	retlw	02Ah
   395  01EA  342A               	retlw	02Ah
   396  01EB  3400               	retlw	0
   397                           opt subtitle "HI-TECH Software Omniscient Code Generator (Lite mode) build 49521"
   398                           
   399                           opt pagewidth 120
   400                           
   401                           	opt lm
   402                           
   403                           	processor	16F1827
   404  000B                     _INTCONbits	set	0xB
   405                           opt subtitle "HI-TECH Software Omniscient Code Generator (Lite mode) build 49521"
   406  0011                     _PIR1bits	set	0x11
   407                           opt subtitle "HI-TECH Software Omniscient Code Generator (Lite mode) build 49521"
   408  000C                     _PORTAbits	set	0xC
   409                           opt subtitle "HI-TECH Software Omniscient Code Generator (Lite mode) build 49521"
   410  001B                     _PR2	set	0x1B
   411                           opt subtitle "HI-TECH Software Omniscient Code Generator (Lite mode) build 49521"
   412  001C                     _T2CON	set	0x1C
   413                           opt subtitle "HI-TECH Software Omniscient Code Generator (Lite mode) build 49521"
   414  006B                     _RB3	set	0x6B
   415                           opt subtitle "HI-TECH Software Omniscient Code Generator (Lite mode) build 49521"
   416  006C                     _RB4	set	0x6C
   417                           opt subtitle "HI-TECH Software Omniscient Code Generator (Lite mode) build 49521"
   418  0095                     _OPTION_REGbits	set	0x95
   419                           opt subtitle "HI-TECH Software Omniscient Code Generator (Lite mode) build 49521"
   420  0099                     _OSCCON	set	0x99
   421                           opt subtitle "HI-TECH Software Omniscient Code Generator (Lite mode) build 49521"
   422  0091                     _PIE1bits	set	0x91
   423                           opt subtitle "HI-TECH Software Omniscient Code Generator (Lite mode) build 49521"
   424  008C                     _TRISA	set	0x8C
   425                           opt subtitle "HI-TECH Software Omniscient Code Generator (Lite mode) build 49521"
   426  008D                     _TRISB	set	0x8D
   427                           opt subtitle "HI-TECH Software Omniscient Code Generator (Lite mode) build 49521"
   428  018C                     _ANSELA	set	0x18C
   429                           opt subtitle "HI-TECH Software Omniscient Code Generator (Lite mode) build 49521"
   430  018D                     _ANSELB	set	0x18D
   431                           opt subtitle "HI-TECH Software Omniscient Code Generator (Lite mode) build 49521"
   432  019F                     _BAUDCON	set	0x19F
   433                           opt subtitle "HI-TECH Software Omniscient Code Generator (Lite mode) build 49521"
   434  0199                     _RCREG	set	0x199
   435                           opt subtitle "HI-TECH Software Omniscient Code Generator (Lite mode) build 49521"
   436  019D                     _RCSTA	set	0x19D
   437                           opt subtitle "HI-TECH Software Omniscient Code Generator (Lite mode) build 49521"
   438  019D                     _RCSTAbits	set	0x19D
   439                           opt subtitle "HI-TECH Software Omniscient Code Generator (Lite mode) build 49521"
   440  019B                     _SPBRG	set	0x19B
   441                           opt subtitle "HI-TECH Software Omniscient Code Generator (Lite mode) build 49521"
   442  019A                     _TXREG	set	0x19A
   443                           opt subtitle "HI-TECH Software Omniscient Code Generator (Lite mode) build 49521"
   444  019E                     _TXSTA	set	0x19E
   445                           opt subtitle "HI-TECH Software Omniscient Code Generator (Lite mode) build 49521"
   446  019E                     _TXSTAbits	set	0x19E
   447                           opt subtitle "HI-TECH Software Omniscient Code Generator (Lite mode) build 49521"
   448  020D                     _WPUB	set	0x20D
   449                           opt subtitle "HI-TECH Software Omniscient Code Generator (Lite mode) build 49521"
   450                           
   451  0000                     __CFG_CPD$OFF equ 0x0
   452                           opt subtitle "HI-TECH Software Omniscient Code Generator (Lite mode) build 49521"
   453  0000                     __CFG_BOREN$ON equ 0x0
   454                           opt subtitle "HI-TECH Software Omniscient Code Generator (Lite mode) build 49521"
   455  0000                     __CFG_IESO$OFF equ 0x0
   456                           opt subtitle "HI-TECH Software Omniscient Code Generator (Lite mode) build 49521"
   457  0000                     __CFG_FOSC$INTOSC equ 0x0
   458                           opt subtitle "HI-TECH Software Omniscient Code Generator (Lite mode) build 49521"
   459  0000                     __CFG_FCMEN$OFF equ 0x0
   460                           opt subtitle "HI-TECH Software Omniscient Code Generator (Lite mode) build 49521"
   461  0000                     __CFG_MCLRE$ON equ 0x0
   462                           opt subtitle "HI-TECH Software Omniscient Code Generator (Lite mode) build 49521"
   463  0000                     __CFG_WDTE$OFF equ 0x0
   464                           opt subtitle "HI-TECH Software Omniscient Code Generator (Lite mode) build 49521"
   465  0000                     __CFG_CP$OFF equ 0x0
   466                           opt subtitle "HI-TECH Software Omniscient Code Generator (Lite mode) build 49521"
   467  0000                     __CFG_PWRTE$ON equ 0x0
   468                           opt subtitle "HI-TECH Software Omniscient Code Generator (Lite mode) build 49521"
   469  0000                     __CFG_CLKOUTEN$ON equ 0x0
   470                           opt subtitle "HI-TECH Software Omniscient Code Generator (Lite mode) build 49521"
   471  0000                     __CFG_PLLEN$ON equ 0x0
   472                           opt subtitle "HI-TECH Software Omniscient Code Generator (Lite mode) build 49521"
   473  0000                     __CFG_WRT$OFF equ 0x0
   474                           opt subtitle "HI-TECH Software Omniscient Code Generator (Lite mode) build 49521"
   475  0000                     __CFG_STVREN$OFF equ 0x0
   476                           opt subtitle "HI-TECH Software Omniscient Code Generator (Lite mode) build 49521"
   477  0000                     __CFG_BORV$LO equ 0x0
   478                           opt subtitle "HI-TECH Software Omniscient Code Generator (Lite mode) build 49521"
   479  0000                     __CFG_LVP$OFF equ 0x0
   480                           opt subtitle "HI-TECH Software Omniscient Code Generator (Lite mode) build 49521"
   481                           
   482                           opt pagewidth 120
   483                           
   484  018E                     start_initialization:
   485                           opt subtitle "HI-TECH Software Omniscient Code Generator (Lite mode) build 49521"
   486                           
   487  018E                     __initialization:
   488  2070                     _Buf  equ     8304	;BIGRAM
   489                           opt subtitle "HI-TECH Software Omniscient Code Generator (Lite mode) build 49521"
   490                           
   491  0070                     __pbssCOMMON:
   492  0070                     _Index:
   493  0070                            ds      2
   494                           opt subtitle "HI-TECH Software Omniscient Code Generator (Lite mode) build 49521"
   495  0072                     _i:
   496  0072                            ds      2
   497                           opt subtitle "HI-TECH Software Omniscient Code Generator (Lite mode) build 49521"
   498  0074                     _ascii:
   499  0074                            ds      1
   500                           opt subtitle "HI-TECH Software Omniscient Code Generator (Lite mode) build 49521"
   501  0075                     _data:
   502  0075                            ds      1
   503                           opt subtitle "HI-TECH Software Omniscient Code Generator (Lite mode) build 49521"
   504                           
   505                           opt pagewidth 120
   506  0045                     __pbssBANK0:
   507  0045                     _rcv:
   508  0045                            ds      1
   509                           opt subtitle "HI-TECH Software Omniscient Code Generator (Lite mode) build 49521"
   510                           
   511                           opt pagewidth 120
   512  0020                     __pdataBANK0:
   513                           opt subtitle "HI-TECH Software Omniscient Code Generator (Lite mode) build 49521"
   514  0020                     _Msg:
   515  0020                            ds      29
   516                           opt subtitle "HI-TECH Software Omniscient Code Generator (Lite mode) build 49521"
   517                           
   518                           opt pagewidth 120
   519                           
   520                           	opt lm
   521  01FA                     clear_ram:
   522  01FA  0064               	clrwdt			;clear the watchdog before getting into this loop
   523  01FB                     clrloop:
   524  01FB  0180               	clrf	indf0		;clear RAM location pointed to by FSR
   525  01FC  3101               	addfsr	0,1
   526  01FD  3001               	movlw	1
   527  01FE  02FE               	subwf	btemp,f
   528  01FF  3000               	movlw	0
   529  0200  3BFF               	subwfb btemp+1,f
   530  0201  087F               	movf btemp+1,w
   531  0202  047E               	iorwf btemp,w
   532  0203  1D03               	skipz
   533  0204  29FB               	goto clrloop	;have we reached the end yet?
   534  0205  3400               	retlw	0		;all done for this memory range, return
   535                           opt subtitle "HI-TECH Software Omniscient Code Generator (Lite mode) build 49521"
   536                           
   537                           opt pagewidth 120
   538  018E  3070               	movlw	low(__pbssBIGRAM)
   539  018F  0084               	movwf	fsr0l
   540  0190  3020               	movlw	high(__pbssBIGRAM)
   541  0191  0085               	movwf	fsr0h
   542  0192  3000               	movlw	low(0100h)
   543  0193  00FE               	movwf	btemp
   544  0194  3001               	movlw	high(0100h)
   545  0195  00FF               	movwf	btemp+1
   546  0196  3181  21FA  3181   	fcall	clear_ram
   547                           opt subtitle "HI-TECH Software Omniscient Code Generator (Lite mode) build 49521"
   548                           
   549                           opt pagewidth 120
   550  0199  01F0               	clrf	((__pbssCOMMON)+0)&07Fh
   551  019A  01F1               	clrf	((__pbssCOMMON)+1)&07Fh
   552  019B  01F2               	clrf	((__pbssCOMMON)+2)&07Fh
   553  019C  01F3               	clrf	((__pbssCOMMON)+3)&07Fh
   554  019D  01F4               	clrf	((__pbssCOMMON)+4)&07Fh
   555  019E  01F5               	clrf	((__pbssCOMMON)+5)&07Fh
   556                           opt subtitle "HI-TECH Software Omniscient Code Generator (Lite mode) build 49521"
   557                           
   558                           opt pagewidth 120
   559  019F  01C5               	clrf	((__pbssBANK0)+0)&07Fh
   560                           opt subtitle "HI-TECH Software Omniscient Code Generator (Lite mode) build 49521"
   561                           
   562  0206                     init_ram:
   563  0206  00FE               	movwf btemp,f
   564  0207                     initloop:
   565  0207  0012               	moviw fsr0++
   566  0208  001E               	movwi fsr1++
   567  0209  3001               	movlw 1
   568  020A  02FE               subwf btemp,f
   569  020B  3000               movlw 0
   570  020C  3BFF               subwfb btemp+1,f
   571  020D  087F               	movf btemp+1,w
   572  020E  047E               	iorwf btemp,w
   573  020F  1D03               	skipz
   574  0210  2A07               	goto initloop
   575  0211  3400               	retlw 0
   576                           opt subtitle "HI-TECH Software Omniscient Code Generator (Lite mode) build 49521"
   577                           
   578                           opt pagewidth 120
   579  01A0  30CF               	movlw low(__pidataBANK0)
   580  01A1  0084               	movwf fsr0l
   581  01A2  3081               	movlw high(__pidataBANK0)|80h
   582  01A3  0085               	movwf fsr0h
   583  01A4  3020               	movlw low(__pdataBANK0)
   584  01A5  0086               	movwf fsr1l
   585  01A6  3000               	movlw high(__pdataBANK0)
   586  01A7  0087               	movwf fsr1h
   587  01A8  3000               	movlw high(01Dh)
   588  01A9  00FF               	movwf btemp+1
   589  01AA  301D               	movlw low(01Dh)
   590  01AB  3182  2206  3181   	fcall init_ram
   591                           opt subtitle "HI-TECH Software Omniscient Code Generator (Lite mode) build 49521"
   592                           
   593                           opt pagewidth 120
   594                           
   595                           	opt lm
   596  01AE                     end_of_initialization:
   597  01AE                     __end_of__initialization:movlb 0
      + 01AE  0020               	movlb	0
   598  01AF  3180  284F         ljmp _main	;jump to C main() function
   599                           opt subtitle "HI-TECH Software Omniscient Code Generator (Lite mode) build 49521"
   600                           
   601  0076                     __pcstackCOMMON:
   602  0076                     ?_Send:	; 0 bytes @ 0x0
   603  0076                     ?_main:	; 0 bytes @ 0x0
   604  0076                     ?_isr:	; 0 bytes @ 0x0
   605  0076                     ??_isr:	; 0 bytes @ 0x0
   606  0076                     	ds	6
   607                           opt subtitle "HI-TECH Software Omniscient Code Generator (Lite mode) build 49521"
   608                           
   609  003D                     __pcstackBANK0:
   610                           opt subtitle "HI-TECH Software Omniscient Code Generator (Lite mode) build 49521"
   611  003D                     ?_Delayms:	; 0 bytes @ 0x0
   612  003D                     ??_Send:	; 0 bytes @ 0x0
   613                           opt subtitle "HI-TECH Software Omniscient Code Generator (Lite mode) build 49521"
   614  003D                     Send@Data:	; 1 bytes @ 0x0
   615                           opt subtitle "HI-TECH Software Omniscient Code Generator (Lite mode) build 49521"
   616  003D                     Delayms@t:	; 2 bytes @ 0x0
   617  003D                     	ds	2
   618  003F                     ??_Delayms:	; 0 bytes @ 0x2
   619  003F                     ??_main:	; 0 bytes @ 0x2
   620  003F                     	ds	6
   621                           opt subtitle "HI-TECH Software Omniscient Code Generator (Lite mode) build 49521"
   622                           
   623                           opt pagewidth 120
   624                           
   625                           	opt lm
   626                           
   627                           	processor	16F1827
   628                           clrc	macro
   629                           	bcf	3,0
   630                           	endm
   631                           clrz	macro
   632                           	bcf	3,2
   633                           	endm
   634                           setc	macro
   635                           	bsf	3,0
   636                           	endm
   637                           setz	macro
   638                           	bsf	3,2
   639                           	endm
   640                           skipc	macro
   641                           	btfss	3,0
   642                           	endm
   643                           skipz	macro
   644                           	btfss	3,2
   645                           	endm
   646                           skipnc	macro
   647                           	btfsc	3,0
   648                           	endm
   649                           skipnz	macro
   650                           	btfsc	3,2
   651                           	endm
   652                           indf	equ	0
   653                           indf0	equ	0
   654                           indf1	equ	1
   655                           pc	equ	2
   656                           pcl	equ	2
   657                           status	equ	3
   658                           fsr0l	equ	4
   659                           fsr0h	equ	5
   660                           fsr1l	equ	6
   661                           fsr1h	equ	7
   662                           bsr	equ	8
   663                           wreg	equ	9
   664                           intcon	equ	11
   665                           c	equ	1
   666                           z	equ	0
   667                           pclath	equ	10
   668                           # 46 "C:\Program Files\Microchip\xc8\v1.12\include\pic16f1827.h"
   669                           INDF0 equ 00h ;# 
   670                           # 65 "C:\Program Files\Microchip\xc8\v1.12\include\pic16f1827.h"
   671                           INDF1 equ 01h ;# 
   672                           # 84 "C:\Program Files\Microchip\xc8\v1.12\include\pic16f1827.h"
   673                           PCL equ 02h ;# 
   674                           # 103 "C:\Program Files\Microchip\xc8\v1.12\include\pic16f1827.h"
   675                           STATUS equ 03h ;# 
   676                           # 166 "C:\Program Files\Microchip\xc8\v1.12\include\pic16f1827.h"
   677                           FSR0L equ 04h ;# 
   678                           # 185 "C:\Program Files\Microchip\xc8\v1.12\include\pic16f1827.h"
   679                           FSR0H equ 05h ;# 
   680                           # 207 "C:\Program Files\Microchip\xc8\v1.12\include\pic16f1827.h"
   681                           FSR1L equ 06h ;# 
   682                           # 226 "C:\Program Files\Microchip\xc8\v1.12\include\pic16f1827.h"
   683                           FSR1H equ 07h ;# 
   684                           # 245 "C:\Program Files\Microchip\xc8\v1.12\include\pic16f1827.h"
   685                           BSR equ 08h ;# 
   686                           # 296 "C:\Program Files\Microchip\xc8\v1.12\include\pic16f1827.h"
   687                           WREG equ 09h ;# 
   688                           # 315 "C:\Program Files\Microchip\xc8\v1.12\include\pic16f1827.h"
   689                           PCLATH equ 0Ah ;# 
   690                           # 334 "C:\Program Files\Microchip\xc8\v1.12\include\pic16f1827.h"
   691                           INTCON equ 0Bh ;# 
   692                           # 411 "C:\Program Files\Microchip\xc8\v1.12\include\pic16f1827.h"
   693                           PORTA equ 0Ch ;# 
   694                           # 472 "C:\Program Files\Microchip\xc8\v1.12\include\pic16f1827.h"
   695                           PORTB equ 0Dh ;# 
   696                           # 533 "C:\Program Files\Microchip\xc8\v1.12\include\pic16f1827.h"
   697                           PIR1 equ 011h ;# 
   698                           # 594 "C:\Program Files\Microchip\xc8\v1.12\include\pic16f1827.h"
   699                           PIR2 equ 012h ;# 
   700                           # 644 "C:\Program Files\Microchip\xc8\v1.12\include\pic16f1827.h"
   701                           PIR3 equ 013h ;# 
   702                           # 683 "C:\Program Files\Microchip\xc8\v1.12\include\pic16f1827.h"
   703                           PIR4 equ 014h ;# 
   704                           # 708 "C:\Program Files\Microchip\xc8\v1.12\include\pic16f1827.h"
   705                           TMR0 equ 015h ;# 
   706                           # 727 "C:\Program Files\Microchip\xc8\v1.12\include\pic16f1827.h"
   707                           TMR1 equ 016h ;# 
   708                           # 733 "C:\Program Files\Microchip\xc8\v1.12\include\pic16f1827.h"
   709                           TMR1L equ 016h ;# 
   710                           # 752 "C:\Program Files\Microchip\xc8\v1.12\include\pic16f1827.h"
   711                           TMR1H equ 017h ;# 
   712                           # 771 "C:\Program Files\Microchip\xc8\v1.12\include\pic16f1827.h"
   713                           T1CON equ 018h ;# 
   714                           # 842 "C:\Program Files\Microchip\xc8\v1.12\include\pic16f1827.h"
   715                           T1GCON equ 019h ;# 
   716                           # 911 "C:\Program Files\Microchip\xc8\v1.12\include\pic16f1827.h"
   717                           TMR2 equ 01Ah ;# 
   718                           # 930 "C:\Program Files\Microchip\xc8\v1.12\include\pic16f1827.h"
   719                           PR2 equ 01Bh ;# 
   720                           # 949 "C:\Program Files\Microchip\xc8\v1.12\include\pic16f1827.h"
   721                           T2CON equ 01Ch ;# 
   722                           # 1019 "C:\Program Files\Microchip\xc8\v1.12\include\pic16f1827.h"
   723                           CPSCON0 equ 01Eh ;# 
   724                           # 1072 "C:\Program Files\Microchip\xc8\v1.12\include\pic16f1827.h"
   725                           CPSCON1 equ 01Fh ;# 
   726                           # 1117 "C:\Program Files\Microchip\xc8\v1.12\include\pic16f1827.h"
   727                           TRISA equ 08Ch ;# 
   728                           # 1178 "C:\Program Files\Microchip\xc8\v1.12\include\pic16f1827.h"
   729                           TRISB equ 08Dh ;# 
   730                           # 1239 "C:\Program Files\Microchip\xc8\v1.12\include\pic16f1827.h"
   731                           PIE1 equ 091h ;# 
   732                           # 1300 "C:\Program Files\Microchip\xc8\v1.12\include\pic16f1827.h"
   733                           PIE2 equ 092h ;# 
   734                           # 1350 "C:\Program Files\Microchip\xc8\v1.12\include\pic16f1827.h"
   735                           PIE3 equ 093h ;# 
   736                           # 1389 "C:\Program Files\Microchip\xc8\v1.12\include\pic16f1827.h"
   737                           PIE4 equ 094h ;# 
   738                           # 1414 "C:\Program Files\Microchip\xc8\v1.12\include\pic16f1827.h"
   739                           OPTION_REG equ 095h ;# 
   740                           # 1496 "C:\Program Files\Microchip\xc8\v1.12\include\pic16f1827.h"
   741                           PCON equ 096h ;# 
   742                           # 1546 "C:\Program Files\Microchip\xc8\v1.12\include\pic16f1827.h"
   743                           WDTCON equ 097h ;# 
   744                           # 1604 "C:\Program Files\Microchip\xc8\v1.12\include\pic16f1827.h"
   745                           OSCTUNE equ 098h ;# 
   746                           # 1661 "C:\Program Files\Microchip\xc8\v1.12\include\pic16f1827.h"
   747                           OSCCON equ 099h ;# 
   748                           # 1732 "C:\Program Files\Microchip\xc8\v1.12\include\pic16f1827.h"
   749                           OSCSTAT equ 09Ah ;# 
   750                           # 1793 "C:\Program Files\Microchip\xc8\v1.12\include\pic16f1827.h"
   751                           ADRES equ 09Bh ;# 
   752                           # 1799 "C:\Program Files\Microchip\xc8\v1.12\include\pic16f1827.h"
   753                           ADRESL equ 09Bh ;# 
   754                           # 1818 "C:\Program Files\Microchip\xc8\v1.12\include\pic16f1827.h"
   755                           ADRESH equ 09Ch ;# 
   756                           # 1837 "C:\Program Files\Microchip\xc8\v1.12\include\pic16f1827.h"
   757                           ADCON0 equ 09Dh ;# 
   758                           # 1916 "C:\Program Files\Microchip\xc8\v1.12\include\pic16f1827.h"
   759                           ADCON1 equ 09Eh ;# 
   760                           # 1987 "C:\Program Files\Microchip\xc8\v1.12\include\pic16f1827.h"
   761                           LATA equ 010Ch ;# 
   762                           # 2043 "C:\Program Files\Microchip\xc8\v1.12\include\pic16f1827.h"
   763                           LATB equ 010Dh ;# 
   764                           # 2104 "C:\Program Files\Microchip\xc8\v1.12\include\pic16f1827.h"
   765                           CM1CON0 equ 0111h ;# 
   766                           # 2160 "C:\Program Files\Microchip\xc8\v1.12\include\pic16f1827.h"
   767                           CM1CON1 equ 0112h ;# 
   768                           # 2225 "C:\Program Files\Microchip\xc8\v1.12\include\pic16f1827.h"
   769                           CM2CON0 equ 0113h ;# 
   770                           # 2281 "C:\Program Files\Microchip\xc8\v1.12\include\pic16f1827.h"
   771                           CM2CON1 equ 0114h ;# 
   772                           # 2346 "C:\Program Files\Microchip\xc8\v1.12\include\pic16f1827.h"
   773                           CMOUT equ 0115h ;# 
   774                           # 2371 "C:\Program Files\Microchip\xc8\v1.12\include\pic16f1827.h"
   775                           BORCON equ 0116h ;# 
   776                           # 2397 "C:\Program Files\Microchip\xc8\v1.12\include\pic16f1827.h"
   777                           FVRCON equ 0117h ;# 
   778                           # 2472 "C:\Program Files\Microchip\xc8\v1.12\include\pic16f1827.h"
   779                           DACCON0 equ 0118h ;# 
   780                           # 2532 "C:\Program Files\Microchip\xc8\v1.12\include\pic16f1827.h"
   781                           DACCON1 equ 0119h ;# 
   782                           # 2583 "C:\Program Files\Microchip\xc8\v1.12\include\pic16f1827.h"
   783                           SRCON0 equ 011Ah ;# 
   784                           # 2653 "C:\Program Files\Microchip\xc8\v1.12\include\pic16f1827.h"
   785                           SRCON1 equ 011Bh ;# 
   786                           # 2714 "C:\Program Files\Microchip\xc8\v1.12\include\pic16f1827.h"
   787                           APFCON0 equ 011Dh ;# 
   788                           # 2775 "C:\Program Files\Microchip\xc8\v1.12\include\pic16f1827.h"
   789                           APFCON1 equ 011Eh ;# 
   790                           # 2794 "C:\Program Files\Microchip\xc8\v1.12\include\pic16f1827.h"
   791                           ANSELA equ 018Ch ;# 
   792                           # 2845 "C:\Program Files\Microchip\xc8\v1.12\include\pic16f1827.h"
   793                           ANSELB equ 018Dh ;# 
   794                           # 2909 "C:\Program Files\Microchip\xc8\v1.12\include\pic16f1827.h"
   795                           EEADR equ 0191h ;# 
   796                           # 2915 "C:\Program Files\Microchip\xc8\v1.12\include\pic16f1827.h"
   797                           EEADRL equ 0191h ;# 
   798                           # 2934 "C:\Program Files\Microchip\xc8\v1.12\include\pic16f1827.h"
   799                           EEADRH equ 0192h ;# 
   800                           # 2953 "C:\Program Files\Microchip\xc8\v1.12\include\pic16f1827.h"
   801                           EEDAT equ 0193h ;# 
   802                           # 2959 "C:\Program Files\Microchip\xc8\v1.12\include\pic16f1827.h"
   803                           EEDATL equ 0193h ;# 
   804                           # 2964 "C:\Program Files\Microchip\xc8\v1.12\include\pic16f1827.h"
   805                           EEDATA equ 0193h ;# 
   806                           # 2996 "C:\Program Files\Microchip\xc8\v1.12\include\pic16f1827.h"
   807                           EEDATH equ 0194h ;# 
   808                           # 3015 "C:\Program Files\Microchip\xc8\v1.12\include\pic16f1827.h"
   809                           EECON1 equ 0195h ;# 
   810                           # 3076 "C:\Program Files\Microchip\xc8\v1.12\include\pic16f1827.h"
   811                           EECON2 equ 0196h ;# 
   812                           # 3095 "C:\Program Files\Microchip\xc8\v1.12\include\pic16f1827.h"
   813                           RCREG equ 0199h ;# 
   814                           # 3114 "C:\Program Files\Microchip\xc8\v1.12\include\pic16f1827.h"
   815                           TXREG equ 019Ah ;# 
   816                           # 3133 "C:\Program Files\Microchip\xc8\v1.12\include\pic16f1827.h"
   817                           SPBRGL equ 019Bh ;# 
   818                           # 3138 "C:\Program Files\Microchip\xc8\v1.12\include\pic16f1827.h"
   819                           SPBRG equ 019Bh ;# 
   820                           # 3170 "C:\Program Files\Microchip\xc8\v1.12\include\pic16f1827.h"
   821                           SPBRGH equ 019Ch ;# 
   822                           # 3189 "C:\Program Files\Microchip\xc8\v1.12\include\pic16f1827.h"
   823                           RCSTA equ 019Dh ;# 
   824                           # 3250 "C:\Program Files\Microchip\xc8\v1.12\include\pic16f1827.h"
   825                           TXSTA equ 019Eh ;# 
   826                           # 3311 "C:\Program Files\Microchip\xc8\v1.12\include\pic16f1827.h"
   827                           BAUDCON equ 019Fh ;# 
   828                           # 3362 "C:\Program Files\Microchip\xc8\v1.12\include\pic16f1827.h"
   829                           WPUA equ 020Ch ;# 
   830                           # 3390 "C:\Program Files\Microchip\xc8\v1.12\include\pic16f1827.h"
   831                           WPUB equ 020Dh ;# 
   832                           # 3459 "C:\Program Files\Microchip\xc8\v1.12\include\pic16f1827.h"
   833                           SSP1BUF equ 0211h ;# 
   834                           # 3464 "C:\Program Files\Microchip\xc8\v1.12\include\pic16f1827.h"
   835                           SSPBUF equ 0211h ;# 
   836                           # 3496 "C:\Program Files\Microchip\xc8\v1.12\include\pic16f1827.h"
   837                           SSP1ADD equ 0212h ;# 
   838                           # 3501 "C:\Program Files\Microchip\xc8\v1.12\include\pic16f1827.h"
   839                           SSPADD equ 0212h ;# 
   840                           # 3533 "C:\Program Files\Microchip\xc8\v1.12\include\pic16f1827.h"
   841                           SSP1MSK equ 0213h ;# 
   842                           # 3538 "C:\Program Files\Microchip\xc8\v1.12\include\pic16f1827.h"
   843                           SSPMSK equ 0213h ;# 
   844                           # 3570 "C:\Program Files\Microchip\xc8\v1.12\include\pic16f1827.h"
   845                           SSP1STAT equ 0214h ;# 
   846                           # 3575 "C:\Program Files\Microchip\xc8\v1.12\include\pic16f1827.h"
   847                           SSPSTAT equ 0214h ;# 
   848                           # 3691 "C:\Program Files\Microchip\xc8\v1.12\include\pic16f1827.h"
   849                           SSP1CON1 equ 0215h ;# 
   850                           # 3696 "C:\Program Files\Microchip\xc8\v1.12\include\pic16f1827.h"
   851                           SSPCON1 equ 0215h ;# 
   852                           # 3700 "C:\Program Files\Microchip\xc8\v1.12\include\pic16f1827.h"
   853                           SSPCON equ 0215h ;# 
   854  004F                     __pmaintext:	;psect for function _main
   855                           opt subtitle "HI-TECH Software Omniscient Code Generator (Lite mode) build 49521"
   856                           
   857                           opt pagewidth 120
   858                           
   859  013F                     	__size_of_main	equ	__end_of_main-_main
   860                           opt subtitle "HI-TECH Software Omniscient Code Generator (Lite mode) build 49521"
   861  004F                     _main:	
   862                           opt subtitle "HI-TECH Software Omniscient Code Generator (Lite mode) build 49521"
   863                           
   864                           opt pagewidth 120
   865                           
   866  004F                     l854:	
   867                           opt subtitle "HI-TECH Software Omniscient Code Generator (Lite mode) build 49521"
   868  004F  30F0               	movlw	(0F0h)
   869  0050  0021               	movlb 1	; select bank1
   870  0051  0099               	movwf	(153)^080h	;volatile
   871                           opt subtitle "HI-TECH Software Omniscient Code Generator (Lite mode) build 49521"
   872                           
   873  0052  3002               	movlw	(02h)
   874  0053  0023               	movlb 3	; select bank3
   875  0054  008C               	movwf	(396)^0180h	;volatile
   876                           opt subtitle "HI-TECH Software Omniscient Code Generator (Lite mode) build 49521"
   877                           
   878  0055                     l856:	
   879                           opt subtitle "HI-TECH Software Omniscient Code Generator (Lite mode) build 49521"
   880  0055  018D               	clrf	(397)^0180h	;volatile
   881                           opt subtitle "HI-TECH Software Omniscient Code Generator (Lite mode) build 49521"
   882                           
   883  0056                     l858:	
   884                           opt subtitle "HI-TECH Software Omniscient Code Generator (Lite mode) build 49521"
   885  0056  3022               	movlw	(022h)
   886  0057  0021               	movlb 1	; select bank1
   887  0058  008C               	movwf	(140)^080h	;volatile
   888                           opt subtitle "HI-TECH Software Omniscient Code Generator (Lite mode) build 49521"
   889                           
   890  0059                     l860:	
   891                           opt subtitle "HI-TECH Software Omniscient Code Generator (Lite mode) build 49521"
   892  0059  30FF               	movlw	(0FFh)
   893  005A  008D               	movwf	(141)^080h	;volatile
   894                           opt subtitle "HI-TECH Software Omniscient Code Generator (Lite mode) build 49521"
   895                           
   896  005B                     l862:	
   897                           opt subtitle "HI-TECH Software Omniscient Code Generator (Lite mode) build 49521"
   898  005B  0020               	movlb 0	; select bank0
   899  005C  120C               	bcf	(12),4	;volatile
   900                           opt subtitle "HI-TECH Software Omniscient Code Generator (Lite mode) build 49521"
   901                           
   902  005D                     l864:	
   903                           opt subtitle "HI-TECH Software Omniscient Code Generator (Lite mode) build 49521"
   904  005D  100C               	bcf	(12),0	;volatile
   905                           opt subtitle "HI-TECH Software Omniscient Code Generator (Lite mode) build 49521"
   906                           
   907  005E                     l866:	
   908                           opt subtitle "HI-TECH Software Omniscient Code Generator (Lite mode) build 49521"
   909  005E  30C8               	movlw	low(0C8h)
   910  005F  00BD               	movwf	(?_Delayms)
   911  0060  3000               	movlw	high(0C8h)
   912  0061  00BE               	movwf	((?_Delayms))+1
   913  0062  3181  21B1  3180   	fcall	_Delayms
   914                           opt subtitle "HI-TECH Software Omniscient Code Generator (Lite mode) build 49521"
   915                           
   916  0065                     l868:	
   917                           opt subtitle "HI-TECH Software Omniscient Code Generator (Lite mode) build 49521"
   918  0065  0020               	movlb 0	; select bank0
   919  0066  140C               	bsf	(12),0	;volatile
   920                           opt subtitle "HI-TECH Software Omniscient Code Generator (Lite mode) build 49521"
   921                           
   922  0067                     l870:	
   923                           opt subtitle "HI-TECH Software Omniscient Code Generator (Lite mode) build 49521"
   924  0067  3018               	movlw	(018h)
   925  0068  0024               	movlb 4	; select bank4
   926  0069  008D               	movwf	(525)^0200h	;volatile
   927                           opt subtitle "HI-TECH Software Omniscient Code Generator (Lite mode) build 49521"
   928                           
   929  006A                     l872:	
   930                           opt subtitle "HI-TECH Software Omniscient Code Generator (Lite mode) build 49521"
   931  006A  0021               	movlb 1	; select bank1
   932  006B  1395               	bcf	(149)^080h,7	;volatile
   933                           opt subtitle "HI-TECH Software Omniscient Code Generator (Lite mode) build 49521"
   934                           
   935  006C                     l874:	
   936                           opt subtitle "HI-TECH Software Omniscient Code Generator (Lite mode) build 49521"
   937  006C  3024               	movlw	(024h)
   938  006D  0023               	movlb 3	; select bank3
   939  006E  009E               	movwf	(414)^0180h	;volatile
   940                           opt subtitle "HI-TECH Software Omniscient Code Generator (Lite mode) build 49521"
   941                           
   942  006F                     l876:	
   943                           opt subtitle "HI-TECH Software Omniscient Code Generator (Lite mode) build 49521"
   944  006F  3090               	movlw	(090h)
   945  0070  009D               	movwf	(413)^0180h	;volatile
   946                           opt subtitle "HI-TECH Software Omniscient Code Generator (Lite mode) build 49521"
   947                           
   948  0071                     l878:	
   949                           opt subtitle "HI-TECH Software Omniscient Code Generator (Lite mode) build 49521"
   950  0071  3008               	movlw	(08h)
   951  0072  009F               	movwf	(415)^0180h	;volatile
   952                           opt subtitle "HI-TECH Software Omniscient Code Generator (Lite mode) build 49521"
   953                           
   954  0073                     l880:	
   955                           opt subtitle "HI-TECH Software Omniscient Code Generator (Lite mode) build 49521"
   956  0073  3044               	movlw	(044h)
   957  0074  009B               	movwf	(411)^0180h	;volatile
   958                           opt subtitle "HI-TECH Software Omniscient Code Generator (Lite mode) build 49521"
   959                           
   960  0075                     l882:	
   961                           opt subtitle "HI-TECH Software Omniscient Code Generator (Lite mode) build 49521"
   962  0075  01F0               	clrf	(_Index)
   963  0076  01F1               	clrf	(_Index+1)
   964                           opt subtitle "HI-TECH Software Omniscient Code Generator (Lite mode) build 49521"
   965                           
   966  0077                     l884:	
   967                           opt subtitle "HI-TECH Software Omniscient Code Generator (Lite mode) build 49521"
   968  0077  3020               	movlw	(020h)
   969  0078  0020               	movlb 0	; select bank0
   970  0079  00BF               	movwf	(??_main+0)+0
   971  007A  083F               	movf	(??_main+0)+0,w
   972  007B  00F4               	movwf	(_ascii)
   973                           opt subtitle "HI-TECH Software Omniscient Code Generator (Lite mode) build 49521"
   974                           
   975  007C                     l886:	
   976                           opt subtitle "HI-TECH Software Omniscient Code Generator (Lite mode) build 49521"
   977  007C  1291               	bcf	(17),5	;volatile
   978                           opt subtitle "HI-TECH Software Omniscient Code Generator (Lite mode) build 49521"
   979                           
   980  007D                     l888:	
   981                           opt subtitle "HI-TECH Software Omniscient Code Generator (Lite mode) build 49521"
   982  007D  0021               	movlb 1	; select bank1
   983  007E  1691               	bsf	(145)^080h,5	;volatile
   984                           opt subtitle "HI-TECH Software Omniscient Code Generator (Lite mode) build 49521"
   985                           
   986  007F                     l890:	
   987                           opt subtitle "HI-TECH Software Omniscient Code Generator (Lite mode) build 49521"
   988  007F  170B               	bsf	(11),6	;volatile
   989                           opt subtitle "HI-TECH Software Omniscient Code Generator (Lite mode) build 49521"
   990                           
   991  0080                     l892:	
   992                           opt subtitle "HI-TECH Software Omniscient Code Generator (Lite mode) build 49521"
   993  0080  178B               	bsf	(11),7	;volatile
   994  0081  2882               	goto	l894
   995                           opt subtitle "HI-TECH Software Omniscient Code Generator (Lite mode) build 49521"
   996                           
   997                           opt pagewidth 120
   998  0082                     l67:	
   999                           opt subtitle "HI-TECH Software Omniscient Code Generator (Lite mode) build 49521"
  1000                           
  1001  0082                     l894:	
  1002                           opt subtitle "HI-TECH Software Omniscient Code Generator (Lite mode) build 49521"
  1003  0082  0871               	movf	(_Index+1),w
  1004  0083  3A80               	xorlw	80h
  1005  0084  00FF               	movwf	btemp+1
  1006  0085  3080               	movlw	(high(01h))^80h
  1007  0086  027F               	subwf	btemp+1,w
  1008  0087  1D03               	skipz
  1009  0088  288B               	goto	u375
  1010  0089  3001               	movlw	low(01h)
  1011  008A  0270               	subwf	(_Index),w
  1012  008B                     u375:
  1013                           opt subtitle "HI-TECH Software Omniscient Code Generator (Lite mode) build 49521"
  1014  008B  1C03               	skipc
  1015  008C  288E               	goto	u371
  1016  008D  288F               	goto	u370
  1017  008E                     u371:
  1018  008E  2930               	goto	l934
  1019  008F                     u370:
  1020                           opt subtitle "HI-TECH Software Omniscient Code Generator (Lite mode) build 49521"
  1021                           
  1022  008F                     l896:	
  1023                           opt subtitle "HI-TECH Software Omniscient Code Generator (Lite mode) build 49521"
  1024  008F  01F2               	clrf	(_i)
  1025  0090  01F3               	clrf	(_i+1)
  1026                           opt subtitle "HI-TECH Software Omniscient Code Generator (Lite mode) build 49521"
  1027                           
  1028  0091  291D               	goto	l930
  1029                           opt subtitle "HI-TECH Software Omniscient Code Generator (Lite mode) build 49521"
  1030  0092                     l70:	
  1031                           opt subtitle "HI-TECH Software Omniscient Code Generator (Lite mode) build 49521"
  1032                           
  1033  0092  28EB               	goto	l928
  1034                           opt subtitle "HI-TECH Software Omniscient Code Generator (Lite mode) build 49521"
  1035                           
  1036                           opt pagewidth 120
  1037  0093                     l72:	
  1038  0093  2894               	goto	l898
  1039                           opt subtitle "HI-TECH Software Omniscient Code Generator (Lite mode) build 49521"
  1040                           
  1041  0094                     l73:	
  1042                           opt subtitle "HI-TECH Software Omniscient Code Generator (Lite mode) build 49521"
  1043                           
  1044  0094                     l898:	
  1045                           opt subtitle "HI-TECH Software Omniscient Code Generator (Lite mode) build 49521"
  1046                           
  1047  0094  300D               	movlw	(0Dh)
  1048  0095  3181  21EC  3180   	fcall	_Send
  1049                           opt subtitle "HI-TECH Software Omniscient Code Generator (Lite mode) build 49521"
  1050                           
  1051  0098  300A               	movlw	(0Ah)
  1052  0099  3181  21EC  3180   	fcall	_Send
  1053                           opt subtitle "HI-TECH Software Omniscient Code Generator (Lite mode) build 49521"
  1054                           
  1055  009C                     l900:	
  1056                           opt subtitle "HI-TECH Software Omniscient Code Generator (Lite mode) build 49521"
  1057  009C  3041               	movlw	(041h)
  1058  009D  0020               	movlb 0	; select bank0
  1059  009E  00BF               	movwf	(??_main+0)+0
  1060  009F  083F               	movf	(??_main+0)+0,w
  1061  00A0  00F5               	movwf	(_data)
  1062                           opt subtitle "HI-TECH Software Omniscient Code Generator (Lite mode) build 49521"
  1063  00A1                     l902:	
  1064  00A1  305B               	movlw	(05Bh)
  1065  00A2  0275               	subwf	(_data),w
  1066  00A3  1C03               	skipc
  1067  00A4  28A6               	goto	u381
  1068  00A5  28A7               	goto	u380
  1069  00A6                     u381:
  1070  00A6  28A9               	goto	l906
  1071  00A7                     u380:
  1072  00A7  291D               	goto	l930
  1073                           opt subtitle "HI-TECH Software Omniscient Code Generator (Lite mode) build 49521"
  1074  00A8                     l904:	
  1075  00A8  291D               	goto	l930
  1076                           opt subtitle "HI-TECH Software Omniscient Code Generator (Lite mode) build 49521"
  1077                           
  1078  00A9                     l74:	
  1079                           opt subtitle "HI-TECH Software Omniscient Code Generator (Lite mode) build 49521"
  1080  00A9                     l906:	
  1081                           opt subtitle "HI-TECH Software Omniscient Code Generator (Lite mode) build 49521"
  1082  00A9  0875               	movf	(_data),w
  1083  00AA  3181  21EC  3180   	fcall	_Send
  1084                           opt subtitle "HI-TECH Software Omniscient Code Generator (Lite mode) build 49521"
  1085                           
  1086  00AD                     l908:	
  1087  00AD  3001               	movlw	(01h)
  1088  00AE  0020               	movlb 0	; select bank0
  1089  00AF  00BF               	movwf	(??_main+0)+0
  1090  00B0  083F               	movf	(??_main+0)+0,w
  1091  00B1  07F5               	addwf	(_data),f
  1092                           opt subtitle "HI-TECH Software Omniscient Code Generator (Lite mode) build 49521"
  1093  00B2                     l910:	
  1094  00B2  305B               	movlw	(05Bh)
  1095  00B3  0275               	subwf	(_data),w
  1096  00B4  1C03               	skipc
  1097  00B5  28B7               	goto	u391
  1098  00B6  28B8               	goto	u390
  1099  00B7                     u391:
  1100  00B7  28A9               	goto	l906
  1101  00B8                     u390:
  1102  00B8  291D               	goto	l930
  1103                           opt subtitle "HI-TECH Software Omniscient Code Generator (Lite mode) build 49521"
  1104  00B9                     l75:	
  1105                           opt subtitle "HI-TECH Software Omniscient Code Generator (Lite mode) build 49521"
  1106                           
  1107  00B9  291D               	goto	l930
  1108                           opt subtitle "HI-TECH Software Omniscient Code Generator (Lite mode) build 49521"
  1109                           
  1110                           opt pagewidth 120
  1111  00BA                     l77:	
  1112  00BA  28BB               	goto	l912
  1113                           opt subtitle "HI-TECH Software Omniscient Code Generator (Lite mode) build 49521"
  1114                           
  1115  00BB                     l78:	
  1116                           opt subtitle "HI-TECH Software Omniscient Code Generator (Lite mode) build 49521"
  1117                           
  1118  00BB                     l912:	
  1119                           opt subtitle "HI-TECH Software Omniscient Code Generator (Lite mode) build 49521"
  1120                           
  1121  00BB  300D               	movlw	(0Dh)
  1122  00BC  3181  21EC  3180   	fcall	_Send
  1123                           opt subtitle "HI-TECH Software Omniscient Code Generator (Lite mode) build 49521"
  1124                           
  1125  00BF  300A               	movlw	(0Ah)
  1126  00C0  3181  21EC  3180   	fcall	_Send
  1127                           opt subtitle "HI-TECH Software Omniscient Code Generator (Lite mode) build 49521"
  1128                           
  1129  00C3                     l914:	
  1130                           opt subtitle "HI-TECH Software Omniscient Code Generator (Lite mode) build 49521"
  1131  00C3  3030               	movlw	(030h)
  1132  00C4  0020               	movlb 0	; select bank0
  1133  00C5  00BF               	movwf	(??_main+0)+0
  1134  00C6  083F               	movf	(??_main+0)+0,w
  1135  00C7  00F5               	movwf	(_data)
  1136                           opt subtitle "HI-TECH Software Omniscient Code Generator (Lite mode) build 49521"
  1137  00C8                     l916:	
  1138  00C8  303A               	movlw	(03Ah)
  1139  00C9  0275               	subwf	(_data),w
  1140  00CA  1C03               	skipc
  1141  00CB  28CD               	goto	u401
  1142  00CC  28CE               	goto	u400
  1143  00CD                     u401:
  1144  00CD  28D0               	goto	l920
  1145  00CE                     u400:
  1146  00CE  291D               	goto	l930
  1147                           opt subtitle "HI-TECH Software Omniscient Code Generator (Lite mode) build 49521"
  1148  00CF                     l918:	
  1149  00CF  291D               	goto	l930
  1150                           opt subtitle "HI-TECH Software Omniscient Code Generator (Lite mode) build 49521"
  1151                           
  1152  00D0                     l79:	
  1153                           opt subtitle "HI-TECH Software Omniscient Code Generator (Lite mode) build 49521"
  1154  00D0                     l920:	
  1155                           opt subtitle "HI-TECH Software Omniscient Code Generator (Lite mode) build 49521"
  1156  00D0  0875               	movf	(_data),w
  1157  00D1  3181  21EC  3180   	fcall	_Send
  1158                           opt subtitle "HI-TECH Software Omniscient Code Generator (Lite mode) build 49521"
  1159                           
  1160  00D4                     l922:	
  1161  00D4  3001               	movlw	(01h)
  1162  00D5  0020               	movlb 0	; select bank0
  1163  00D6  00BF               	movwf	(??_main+0)+0
  1164  00D7  083F               	movf	(??_main+0)+0,w
  1165  00D8  07F5               	addwf	(_data),f
  1166                           opt subtitle "HI-TECH Software Omniscient Code Generator (Lite mode) build 49521"
  1167  00D9                     l924:	
  1168  00D9  303A               	movlw	(03Ah)
  1169  00DA  0275               	subwf	(_data),w
  1170  00DB  1C03               	skipc
  1171  00DC  28DE               	goto	u411
  1172  00DD  28DF               	goto	u410
  1173  00DE                     u411:
  1174  00DE  28D0               	goto	l920
  1175  00DF                     u410:
  1176  00DF  291D               	goto	l930
  1177                           opt subtitle "HI-TECH Software Omniscient Code Generator (Lite mode) build 49521"
  1178  00E0                     l80:	
  1179                           opt subtitle "HI-TECH Software Omniscient Code Generator (Lite mode) build 49521"
  1180                           
  1181  00E0  291D               	goto	l930
  1182                           opt subtitle "HI-TECH Software Omniscient Code Generator (Lite mode) build 49521"
  1183                           
  1184                           opt pagewidth 120
  1185  00E1                     l81:	
  1186                           opt subtitle "HI-TECH Software Omniscient Code Generator (Lite mode) build 49521"
  1187                           
  1188  00E1  150C               	bsf	(12),2	;volatile
  1189                           opt subtitle "HI-TECH Software Omniscient Code Generator (Lite mode) build 49521"
  1190                           
  1191  00E2  291D               	goto	l930
  1192                           opt subtitle "HI-TECH Software Omniscient Code Generator (Lite mode) build 49521"
  1193                           
  1194                           opt pagewidth 120
  1195  00E3                     l82:	
  1196                           opt subtitle "HI-TECH Software Omniscient Code Generator (Lite mode) build 49521"
  1197                           
  1198  00E3  110C               	bcf	(12),2	;volatile
  1199                           opt subtitle "HI-TECH Software Omniscient Code Generator (Lite mode) build 49521"
  1200                           
  1201  00E4  291D               	goto	l930
  1202                           opt subtitle "HI-TECH Software Omniscient Code Generator (Lite mode) build 49521"
  1203                           
  1204                           opt pagewidth 120
  1205  00E5                     l83:	
  1206                           opt subtitle "HI-TECH Software Omniscient Code Generator (Lite mode) build 49521"
  1207                           
  1208  00E5  158C               	bsf	(12),3	;volatile
  1209                           opt subtitle "HI-TECH Software Omniscient Code Generator (Lite mode) build 49521"
  1210                           
  1211  00E6  291D               	goto	l930
  1212                           opt subtitle "HI-TECH Software Omniscient Code Generator (Lite mode) build 49521"
  1213                           
  1214                           opt pagewidth 120
  1215  00E7                     l84:	
  1216                           opt subtitle "HI-TECH Software Omniscient Code Generator (Lite mode) build 49521"
  1217                           
  1218  00E7  118C               	bcf	(12),3	;volatile
  1219                           opt subtitle "HI-TECH Software Omniscient Code Generator (Lite mode) build 49521"
  1220                           
  1221  00E8  291D               	goto	l930
  1222                           opt subtitle "HI-TECH Software Omniscient Code Generator (Lite mode) build 49521"
  1223                           
  1224                           opt pagewidth 120
  1225  00E9                     l85:	
  1226  00E9  291D               	goto	l930
  1227                           opt subtitle "HI-TECH Software Omniscient Code Generator (Lite mode) build 49521"
  1228                           
  1229  00EA                     l926:	
  1230                           opt subtitle "HI-TECH Software Omniscient Code Generator (Lite mode) build 49521"
  1231  00EA  291D               	goto	l930
  1232                           opt subtitle "HI-TECH Software Omniscient Code Generator (Lite mode) build 49521"
  1233                           
  1234  00EB                     l71:	
  1235                           opt subtitle "HI-TECH Software Omniscient Code Generator (Lite mode) build 49521"
  1236  00EB                     l928:	
  1237  00EB  0873               	movf	(_i+1),w
  1238  00EC  0020               	movlb 0	; select bank0
  1239  00ED  00C0               	movwf	(??_main+0)+0+1
  1240  00EE  0872               	movf	(_i),w
  1241  00EF  00BF               	movwf	(??_main+0)+0
  1242  00F0  3001               	movlw	(01h)
  1243  00F1  07F2               	addwf	(_i),f
  1244  00F2  1803               	skipnc
  1245  00F3  0AF3               	incf	(_i+1),f
  1246  00F4  3070               	movlw	low(8304)
  1247  00F5  00C1               	movwf	(??_main+2)+0
  1248  00F6  3020               	movlw	high(8304)
  1249  00F7  00C2               	movwf	(??_main+2)+0+1
  1250  00F8  083F               	movf	0+(??_main+0)+0,w
  1251  00F9  0741               	addwf	0+(??_main+2)+0,w
  1252  00FA  00C3               	movwf	(??_main+4)+0
  1253  00FB  0840               	movf	1+(??_main+0)+0,w
  1254  00FC  3D42               	addwfc	1+(??_main+2)+0,w
  1255  00FD  00C4               	movwf	1+(??_main+4)+0
  1256  00FE  0843               	movf	0+(??_main+4)+0,w
  1257  00FF  0086               	movwf	fsr1l
  1258  0100  0844               	movf	1+(??_main+4)+0,w
  1259  0101  0087               	movwf	fsr1h
  1260                           opt subtitle "HI-TECH Software Omniscient Code Generator (Lite mode) build 49521"
  1261  0102  0801               	movf	indf1,w
  1262                           opt subtitle "HI-TECH Software Omniscient Code Generator (Lite mode) build 49521"
  1263                           
  1264                           opt pagewidth 120
  1265                           
  1266                           	opt lm
  1267                           
  1268                           	processor	16F1827
  1269                           clrc	macro
  1270                           	bcf	3,0
  1271                           	endm
  1272  0103  3A31               	xorlw	49^0	; case 49
  1273  0104  1903               	skipnz
  1274  0105  28E1               	goto	l81
  1275  0106  3A03               	xorlw	50^49	; case 50
  1276  0107  1903               	skipnz
  1277  0108  28E3               	goto	l82
  1278  0109  3A01               	xorlw	51^50	; case 51
  1279  010A  1903               	skipnz
  1280  010B  28E5               	goto	l83
  1281  010C  3A07               	xorlw	52^51	; case 52
  1282  010D  1903               	skipnz
  1283  010E  28E7               	goto	l84
  1284  010F  3A75               	xorlw	65^52	; case 65
  1285  0110  1903               	skipnz
  1286  0111  2894               	goto	l898
  1287  0112  3A0F               	xorlw	78^65	; case 78
  1288  0113  1903               	skipnz
  1289  0114  28BB               	goto	l912
  1290  0115  3A2F               	xorlw	97^78	; case 97
  1291  0116  1903               	skipnz
  1292  0117  2894               	goto	l898
  1293  0118  3A0F               	xorlw	110^97	; case 110
  1294  0119  1903               	skipnz
  1295  011A  28BB               	goto	l912
  1296  011B  291D               	goto	l930
  1297                           opt subtitle "HI-TECH Software Omniscient Code Generator (Lite mode) build 49521"
  1298                           
  1299                           opt pagewidth 120
  1300                           
  1301  011C                     l76:	
  1302  011C  291D               	goto	l930
  1303                           opt subtitle "HI-TECH Software Omniscient Code Generator (Lite mode) build 49521"
  1304                           
  1305  011D                     l69:	
  1306                           opt subtitle "HI-TECH Software Omniscient Code Generator (Lite mode) build 49521"
  1307                           
  1308  011D                     l930:	
  1309  011D  0873               	movf	(_i+1),w
  1310  011E  3A80               	xorlw	80h
  1311  011F  0020               	movlb 0	; select bank0
  1312  0120  00BF               	movwf	(??_main+0)+0
  1313  0121  0871               	movf	(_Index+1),w
  1314  0122  3A80               	xorlw	80h
  1315  0123  023F               	subwf	(??_main+0)+0,w
  1316  0124  1D03               	skipz
  1317  0125  2928               	goto	u425
  1318  0126  0870               	movf	(_Index),w
  1319  0127  0272               	subwf	(_i),w
  1320  0128                     u425:
  1321                           opt subtitle "HI-TECH Software Omniscient Code Generator (Lite mode) build 49521"
  1322  0128  1C03               	skipc
  1323  0129  292B               	goto	u421
  1324  012A  292C               	goto	u420
  1325  012B                     u421:
  1326  012B  28EB               	goto	l928
  1327  012C                     u420:
  1328  012C  292D               	goto	l932
  1329                           opt subtitle "HI-TECH Software Omniscient Code Generator (Lite mode) build 49521"
  1330  012D                     l86:	
  1331                           opt subtitle "HI-TECH Software Omniscient Code Generator (Lite mode) build 49521"
  1332                           
  1333  012D                     l932:	
  1334                           opt subtitle "HI-TECH Software Omniscient Code Generator (Lite mode) build 49521"
  1335                           
  1336  012D  01F0               	clrf	(_Index)
  1337  012E  01F1               	clrf	(_Index+1)
  1338  012F  2930               	goto	l934
  1339                           opt subtitle "HI-TECH Software Omniscient Code Generator (Lite mode) build 49521"
  1340                           
  1341  0130                     l68:	
  1342                           opt subtitle "HI-TECH Software Omniscient Code Generator (Lite mode) build 49521"
  1343                           
  1344  0130                     l934:	
  1345                           opt subtitle "HI-TECH Software Omniscient Code Generator (Lite mode) build 49521"
  1346                           
  1347  0130  0020               	movlb 0	; select bank0
  1348  0131  198D               	btfsc	(107/8),(107)&7	;volatile
  1349  0132  2934               	goto	u431
  1350  0133  2935               	goto	u430
  1351  0134                     u431:
  1352  0134  2962               	goto	l952
  1353  0135                     u430:
  1354                           opt subtitle "HI-TECH Software Omniscient Code Generator (Lite mode) build 49521"
  1355                           
  1356  0135                     l936:	
  1357                           opt subtitle "HI-TECH Software Omniscient Code Generator (Lite mode) build 49521"
  1358  0135  300D               	movlw	(0Dh)
  1359  0136  3181  21EC  3180   	fcall	_Send
  1360                           opt subtitle "HI-TECH Software Omniscient Code Generator (Lite mode) build 49521"
  1361                           
  1362  0139  300A               	movlw	(0Ah)
  1363  013A  3181  21EC  3180   	fcall	_Send
  1364                           opt subtitle "HI-TECH Software Omniscient Code Generator (Lite mode) build 49521"
  1365                           
  1366  013D                     l938:	
  1367                           opt subtitle "HI-TECH Software Omniscient Code Generator (Lite mode) build 49521"
  1368  013D  3040               	movlw	(040h)
  1369  013E  0020               	movlb 0	; select bank0
  1370  013F  00BF               	movwf	(??_main+0)+0
  1371  0140  083F               	movf	(??_main+0)+0,w
  1372  0141  00F4               	movwf	(_ascii)
  1373                           opt subtitle "HI-TECH Software Omniscient Code Generator (Lite mode) build 49521"
  1374  0142                     l940:	
  1375  0142  3080               	movlw	(080h)
  1376  0143  0274               	subwf	(_ascii),w
  1377  0144  1C03               	skipc
  1378  0145  2947               	goto	u441
  1379  0146  2948               	goto	u440
  1380  0147                     u441:
  1381  0147  294A               	goto	l944
  1382  0148                     u440:
  1383  0148  295A               	goto	l950
  1384                           opt subtitle "HI-TECH Software Omniscient Code Generator (Lite mode) build 49521"
  1385  0149                     l942:	
  1386  0149  295A               	goto	l950
  1387                           opt subtitle "HI-TECH Software Omniscient Code Generator (Lite mode) build 49521"
  1388                           
  1389  014A                     l88:	
  1390                           opt subtitle "HI-TECH Software Omniscient Code Generator (Lite mode) build 49521"
  1391  014A                     l944:	
  1392                           opt subtitle "HI-TECH Software Omniscient Code Generator (Lite mode) build 49521"
  1393  014A  0874               	movf	(_ascii),w
  1394  014B  3181  21EC  3180   	fcall	_Send
  1395                           opt subtitle "HI-TECH Software Omniscient Code Generator (Lite mode) build 49521"
  1396                           
  1397  014E                     l946:	
  1398  014E  3001               	movlw	(01h)
  1399  014F  0020               	movlb 0	; select bank0
  1400  0150  00BF               	movwf	(??_main+0)+0
  1401  0151  083F               	movf	(??_main+0)+0,w
  1402  0152  07F4               	addwf	(_ascii),f
  1403                           opt subtitle "HI-TECH Software Omniscient Code Generator (Lite mode) build 49521"
  1404  0153                     l948:	
  1405  0153  3080               	movlw	(080h)
  1406  0154  0274               	subwf	(_ascii),w
  1407  0155  1C03               	skipc
  1408  0156  2958               	goto	u451
  1409  0157  2959               	goto	u450
  1410  0158                     u451:
  1411  0158  294A               	goto	l944
  1412  0159                     u450:
  1413  0159  295A               	goto	l950
  1414                           opt subtitle "HI-TECH Software Omniscient Code Generator (Lite mode) build 49521"
  1415  015A                     l89:	
  1416                           opt subtitle "HI-TECH Software Omniscient Code Generator (Lite mode) build 49521"
  1417                           
  1418  015A                     l950:	
  1419                           opt subtitle "HI-TECH Software Omniscient Code Generator (Lite mode) build 49521"
  1420  015A  3064               	movlw	low(064h)
  1421  015B  00BD               	movwf	(?_Delayms)
  1422  015C  3000               	movlw	high(064h)
  1423  015D  00BE               	movwf	((?_Delayms))+1
  1424  015E  3181  21B1  3180   	fcall	_Delayms
  1425  0161  2962               	goto	l952
  1426                           opt subtitle "HI-TECH Software Omniscient Code Generator (Lite mode) build 49521"
  1427                           
  1428  0162                     l87:	
  1429                           opt subtitle "HI-TECH Software Omniscient Code Generator (Lite mode) build 49521"
  1430                           
  1431  0162                     l952:	
  1432                           opt subtitle "HI-TECH Software Omniscient Code Generator (Lite mode) build 49521"
  1433                           
  1434  0162  0020               	movlb 0	; select bank0
  1435  0163  1A0D               	btfsc	(108/8),(108)&7	;volatile
  1436  0164  2966               	goto	u461
  1437  0165  2967               	goto	u460
  1438  0166                     u461:
  1439  0166  2882               	goto	l894
  1440  0167                     u460:
  1441                           opt subtitle "HI-TECH Software Omniscient Code Generator (Lite mode) build 49521"
  1442                           
  1443  0167                     l954:	
  1444                           opt subtitle "HI-TECH Software Omniscient Code Generator (Lite mode) build 49521"
  1445  0167  01F2               	clrf	(_i)
  1446  0168  01F3               	clrf	(_i+1)
  1447                           opt subtitle "HI-TECH Software Omniscient Code Generator (Lite mode) build 49521"
  1448                           
  1449  0169  2977               	goto	l960
  1450                           opt subtitle "HI-TECH Software Omniscient Code Generator (Lite mode) build 49521"
  1451  016A                     l92:	
  1452                           opt subtitle "HI-TECH Software Omniscient Code Generator (Lite mode) build 49521"
  1453                           
  1454  016A                     l956:	
  1455                           opt subtitle "HI-TECH Software Omniscient Code Generator (Lite mode) build 49521"
  1456  016A  0872               	movf	(_i),w
  1457  016B  3E20               	addlw	_Msg&0ffh
  1458  016C  0086               	movwf	fsr1l
  1459  016D  0187               	clrf fsr1h	
  1460                           opt subtitle "HI-TECH Software Omniscient Code Generator (Lite mode) build 49521"
  1461  016E  0801               	movf	indf1,w
  1462  016F  3181  21EC  3180   	fcall	_Send
  1463                           opt subtitle "HI-TECH Software Omniscient Code Generator (Lite mode) build 49521"
  1464  0172                     l958:	
  1465  0172  3001               	movlw	low(01h)
  1466  0173  07F2               	addwf	(_i),f
  1467  0174  3000               	movlw	high(01h)
  1468  0175  3DF3               	addwfc	(_i+1),f
  1469  0176  2977               	goto	l960
  1470                           opt subtitle "HI-TECH Software Omniscient Code Generator (Lite mode) build 49521"
  1471  0177                     l91:	
  1472                           opt subtitle "HI-TECH Software Omniscient Code Generator (Lite mode) build 49521"
  1473                           
  1474  0177                     l960:	
  1475  0177  0872               	movf	(_i),w
  1476  0178  3E20               	addlw	_Msg&0ffh
  1477  0179  0086               	movwf	fsr1l
  1478  017A  0187               	clrf fsr1h	
  1479                           opt subtitle "HI-TECH Software Omniscient Code Generator (Lite mode) build 49521"
  1480  017B  0881               	movf	indf1,f
  1481  017C  1D03               	skipz
  1482  017D  297F               	goto	u471
  1483  017E  2980               	goto	u470
  1484  017F                     u471:
  1485  017F  296A               	goto	l956
  1486  0180                     u470:
  1487  0180  2981               	goto	l962
  1488                           opt subtitle "HI-TECH Software Omniscient Code Generator (Lite mode) build 49521"
  1489  0181                     l93:	
  1490                           opt subtitle "HI-TECH Software Omniscient Code Generator (Lite mode) build 49521"
  1491                           
  1492  0181                     l962:	
  1493                           opt subtitle "HI-TECH Software Omniscient Code Generator (Lite mode) build 49521"
  1494  0181  3032               	movlw	low(032h)
  1495  0182  0020               	movlb 0	; select bank0
  1496  0183  00BD               	movwf	(?_Delayms)
  1497  0184  3000               	movlw	high(032h)
  1498  0185  00BE               	movwf	((?_Delayms))+1
  1499  0186  3181  21B1  3180   	fcall	_Delayms
  1500  0189  2882               	goto	l894
  1501                           opt subtitle "HI-TECH Software Omniscient Code Generator (Lite mode) build 49521"
  1502                           
  1503  018A                     l90:	
  1504  018A  2882               	goto	l894
  1505                           opt subtitle "HI-TECH Software Omniscient Code Generator (Lite mode) build 49521"
  1506                           
  1507  018B                     l94:	
  1508                           opt subtitle "HI-TECH Software Omniscient Code Generator (Lite mode) build 49521"
  1509  018B  2882               	goto	l894
  1510                           opt subtitle "HI-TECH Software Omniscient Code Generator (Lite mode) build 49521"
  1511  018C                     l95:	
  1512                           opt subtitle "HI-TECH Software Omniscient Code Generator (Lite mode) build 49521"
  1513                           
  1514  018C                     l96:	
  1515                           opt subtitle "HI-TECH Software Omniscient Code Generator (Lite mode) build 49521"
  1516  018C  3180  284D         	ljmp	start
  1517                           opt subtitle "HI-TECH Software Omniscient Code Generator (Lite mode) build 49521"
  1518                           
  1519  018E                     	__end_of_main:
  1520                           opt subtitle "HI-TECH Software Omniscient Code Generator (Lite mode) build 49521"
  1521                           
  1522                           opt pagewidth 120
  1523                           
  1524                           	opt lm
  1525                           
  1526                           	processor	16F1827
  1527                           clrc	macro
  1528                           	bcf	3,0
  1529                           	endm
  1530                           clrz	macro
  1531                           	bcf	3,2
  1532                           	endm
  1533                           setc	macro
  1534                           	bsf	3,0
  1535                           	endm
  1536                           setz	macro
  1537                           	bsf	3,2
  1538                           	endm
  1539                           skipc	macro
  1540                           	btfss	3,0
  1541                           	endm
  1542                           skipz	macro
  1543                           	btfss	3,2
  1544                           	endm
  1545                           skipnc	macro
  1546                           	btfsc	3,0
  1547                           	endm
  1548                           skipnz	macro
  1549                           	btfsc	3,2
  1550                           	endm
  1551                           indf	equ	0
  1552                           indf0	equ	0
  1553                           indf1	equ	1
  1554  01B1                     __ptext143:	;psect for function _Delayms
  1555                           opt subtitle "HI-TECH Software Omniscient Code Generator (Lite mode) build 49521"
  1556                           
  1557                           opt pagewidth 120
  1558                           
  1559  001E                     	__size_of_Delayms	equ	__end_of_Delayms-_Delayms
  1560                           opt subtitle "HI-TECH Software Omniscient Code Generator (Lite mode) build 49521"
  1561  01B1                     _Delayms:	
  1562                           opt subtitle "HI-TECH Software Omniscient Code Generator (Lite mode) build 49521"
  1563                           
  1564                           opt pagewidth 120
  1565                           
  1566  01B1                     l964:	
  1567                           opt subtitle "HI-TECH Software Omniscient Code Generator (Lite mode) build 49521"
  1568  01B1  0020               	movlb 0	; select bank0
  1569  01B2  1091               	bcf	(17),1	;volatile
  1570                           opt subtitle "HI-TECH Software Omniscient Code Generator (Lite mode) build 49521"
  1571                           
  1572  01B3                     l966:	
  1573                           opt subtitle "HI-TECH Software Omniscient Code Generator (Lite mode) build 49521"
  1574  01B3  307D               	movlw	(07Dh)
  1575  01B4  009B               	movwf	(27)	;volatile
  1576                           opt subtitle "HI-TECH Software Omniscient Code Generator (Lite mode) build 49521"
  1577                           
  1578  01B5  3007               	movlw	(07h)
  1579  01B6  009C               	movwf	(28)	;volatile
  1580                           opt subtitle "HI-TECH Software Omniscient Code Generator (Lite mode) build 49521"
  1581                           
  1582  01B7  29BF               	goto	l968
  1583                           opt subtitle "HI-TECH Software Omniscient Code Generator (Lite mode) build 49521"
  1584  01B8                     l116:	
  1585                           opt subtitle "HI-TECH Software Omniscient Code Generator (Lite mode) build 49521"
  1586                           
  1587  01B8  29B9               	goto	l117
  1588                           opt subtitle "HI-TECH Software Omniscient Code Generator (Lite mode) build 49521"
  1589  01B9                     l118:	
  1590                           opt subtitle "HI-TECH Software Omniscient Code Generator (Lite mode) build 49521"
  1591  01B9                     l117:	
  1592  01B9  1C91               	btfss	(17),1	;volatile
  1593  01BA  29BC               	goto	u481
  1594  01BB  29BD               	goto	u480
  1595  01BC                     u481:
  1596  01BC  29B9               	goto	l117
  1597  01BD                     u480:
  1598                           opt subtitle "HI-TECH Software Omniscient Code Generator (Lite mode) build 49521"
  1599  01BD                     l119:	
  1600                           opt subtitle "HI-TECH Software Omniscient Code Generator (Lite mode) build 49521"
  1601                           
  1602  01BD  1091               	bcf	(17),1	;volatile
  1603  01BE  29BF               	goto	l968
  1604                           opt subtitle "HI-TECH Software Omniscient Code Generator (Lite mode) build 49521"
  1605                           
  1606  01BF                     l115:	
  1607                           opt subtitle "HI-TECH Software Omniscient Code Generator (Lite mode) build 49521"
  1608                           
  1609  01BF                     l968:	
  1610  01BF  3001               	movlw	low(01h)
  1611  01C0  02BD               	subwf	(Delayms@t),f
  1612  01C1  3000               	movlw	high(01h)
  1613  01C2  3BBE               	subwfb	(Delayms@t+1),f
  1614  01C3  30FF               	movlw	high(0FFFFh)
  1615  01C4  063E               	xorwf	((Delayms@t+1)),w
  1616  01C5  1D03               	skipz
  1617  01C6  29C9               	goto	u495
  1618  01C7  30FF               	movlw	low(0FFFFh)
  1619  01C8  063D               	xorwf	((Delayms@t)),w
  1620  01C9                     u495:
  1621                           opt subtitle "HI-TECH Software Omniscient Code Generator (Lite mode) build 49521"
  1622  01C9  1D03               	skipz
  1623  01CA  29CC               	goto	u491
  1624  01CB  29CD               	goto	u490
  1625  01CC                     u491:
  1626  01CC  29B9               	goto	l117
  1627  01CD                     u490:
  1628  01CD  29CE               	goto	l121
  1629                           opt subtitle "HI-TECH Software Omniscient Code Generator (Lite mode) build 49521"
  1630  01CE                     l120:	
  1631                           opt subtitle "HI-TECH Software Omniscient Code Generator (Lite mode) build 49521"
  1632                           
  1633  01CE                     l121:	
  1634  01CE  0008               	return
  1635                           opt subtitle "HI-TECH Software Omniscient Code Generator (Lite mode) build 49521"
  1636                           
  1637  01CF                     	__end_of_Delayms:
  1638                           opt subtitle "HI-TECH Software Omniscient Code Generator (Lite mode) build 49521"
  1639                           
  1640                           opt pagewidth 120
  1641                           
  1642                           	opt lm
  1643                           
  1644                           	processor	16F1827
  1645                           clrc	macro
  1646                           	bcf	3,0
  1647                           	endm
  1648                           clrz	macro
  1649                           	bcf	3,2
  1650                           	endm
  1651                           setc	macro
  1652                           	bsf	3,0
  1653                           	endm
  1654                           setz	macro
  1655                           	bsf	3,2
  1656                           	endm
  1657                           skipc	macro
  1658                           	btfss	3,0
  1659                           	endm
  1660                           skipz	macro
  1661                           	btfss	3,2
  1662                           	endm
  1663                           skipnc	macro
  1664                           	btfsc	3,0
  1665                           	endm
  1666                           skipnz	macro
  1667                           	btfsc	3,2
  1668                           	endm
  1669                           indf	equ	0
  1670                           indf0	equ	0
  1671                           indf1	equ	1
  1672  01EC                     __ptext144:	;psect for function _Send
  1673                           opt subtitle "HI-TECH Software Omniscient Code Generator (Lite mode) build 49521"
  1674                           
  1675                           opt pagewidth 120
  1676                           
  1677  000E                     	__size_of_Send	equ	__end_of_Send-_Send
  1678                           opt subtitle "HI-TECH Software Omniscient Code Generator (Lite mode) build 49521"
  1679  01EC                     _Send:	
  1680                           opt subtitle "HI-TECH Software Omniscient Code Generator (Lite mode) build 49521"
  1681                           
  1682                           opt pagewidth 120
  1683  01EC  0020               	movlb 0	; select bank0
  1684  01ED  00BD               	movwf	(Send@Data)
  1685                           opt subtitle "HI-TECH Software Omniscient Code Generator (Lite mode) build 49521"
  1686                           
  1687  01EE                     l970:	
  1688                           opt subtitle "HI-TECH Software Omniscient Code Generator (Lite mode) build 49521"
  1689  01EE  29EF               	goto	l109
  1690                           opt subtitle "HI-TECH Software Omniscient Code Generator (Lite mode) build 49521"
  1691  01EF                     l110:	
  1692                           opt subtitle "HI-TECH Software Omniscient Code Generator (Lite mode) build 49521"
  1693  01EF                     l109:	
  1694  01EF  0023               	movlb 3	; select bank3
  1695  01F0  1C9E               	btfss	(414)^0180h,1	;volatile
  1696  01F1  29F3               	goto	u501
  1697  01F2  29F4               	goto	u500
  1698  01F3                     u501:
  1699  01F3  29EF               	goto	l109
  1700  01F4                     u500:
  1701  01F4  29F5               	goto	l972
  1702                           opt subtitle "HI-TECH Software Omniscient Code Generator (Lite mode) build 49521"
  1703  01F5                     l111:	
  1704                           opt subtitle "HI-TECH Software Omniscient Code Generator (Lite mode) build 49521"
  1705                           
  1706  01F5                     l972:	
  1707                           opt subtitle "HI-TECH Software Omniscient Code Generator (Lite mode) build 49521"
  1708  01F5  0020               	movlb 0	; select bank0
  1709  01F6  083D               	movf	(Send@Data),w
  1710  01F7  0023               	movlb 3	; select bank3
  1711  01F8  009A               	movwf	(410)^0180h	;volatile
  1712                           opt subtitle "HI-TECH Software Omniscient Code Generator (Lite mode) build 49521"
  1713                           
  1714  01F9                     l112:	
  1715  01F9  0008               	return
  1716                           opt subtitle "HI-TECH Software Omniscient Code Generator (Lite mode) build 49521"
  1717                           
  1718  01FA                     	__end_of_Send:
  1719                           opt subtitle "HI-TECH Software Omniscient Code Generator (Lite mode) build 49521"
  1720                           
  1721                           opt pagewidth 120
  1722                           
  1723                           	opt lm
  1724                           
  1725                           	processor	16F1827
  1726                           clrc	macro
  1727                           	bcf	3,0
  1728                           	endm
  1729                           clrz	macro
  1730                           	bcf	3,2
  1731                           	endm
  1732                           setc	macro
  1733                           	bsf	3,0
  1734                           	endm
  1735                           setz	macro
  1736                           	bsf	3,2
  1737                           	endm
  1738                           skipc	macro
  1739                           	btfss	3,0
  1740                           	endm
  1741                           skipz	macro
  1742                           	btfss	3,2
  1743                           	endm
  1744                           skipnc	macro
  1745                           	btfsc	3,0
  1746                           	endm
  1747                           skipnz	macro
  1748                           	btfsc	3,2
  1749                           	endm
  1750                           indf	equ	0
  1751                           indf0	equ	0
  1752  0004                     __pintentry:
  1753                           opt subtitle "HI-TECH Software Omniscient Code Generator (Lite mode) build 49521"
  1754                           
  1755                           opt pagewidth 120
  1756                           
  1757  0049                     	__size_of_isr	equ	__end_of_isr-_isr
  1758                           opt subtitle "HI-TECH Software Omniscient Code Generator (Lite mode) build 49521"
  1759  0004                     _isr:	
  1760                           opt subtitle "HI-TECH Software Omniscient Code Generator (Lite mode) build 49521"
  1761                           
  1762                           opt pagewidth 120
  1763  0004  3180               	pagesel	$
  1764  0005  0020               	movlb 0	; select bank0
  1765  0006  087F               	movf	btemp+1,w
  1766  0007  00FB               	movwf	(??_isr+5)
  1767                           opt subtitle "HI-TECH Software Omniscient Code Generator (Lite mode) build 49521"
  1768                           
  1769  0008                     i1l836:	
  1770                           opt subtitle "HI-TECH Software Omniscient Code Generator (Lite mode) build 49521"
  1771  0008  1E91               	btfss	(17),5	;volatile
  1772  0009  280B               	goto	u33_21
  1773  000A  280C               	goto	u33_20
  1774  000B                     u33_21:
  1775  000B  2849               	goto	i1l106
  1776  000C                     u33_20:
  1777                           opt subtitle "HI-TECH Software Omniscient Code Generator (Lite mode) build 49521"
  1778                           
  1779  000C                     i1l838:	
  1780                           opt subtitle "HI-TECH Software Omniscient Code Generator (Lite mode) build 49521"
  1781  000C  1291               	bcf	(17),5	;volatile
  1782                           opt subtitle "HI-TECH Software Omniscient Code Generator (Lite mode) build 49521"
  1783                           
  1784  000D  0023               	movlb 3	; select bank3
  1785  000E  189D               	btfsc	(413)^0180h,1	;volatile
  1786  000F  2811               	goto	u34_21
  1787  0010  2812               	goto	u34_20
  1788  0011                     u34_21:
  1789  0011  2817               	goto	i1l842
  1790  0012                     u34_20:
  1791                           opt subtitle "HI-TECH Software Omniscient Code Generator (Lite mode) build 49521"
  1792  0012                     i1l840:	
  1793  0012  1D1D               	btfss	(413)^0180h,2	;volatile
  1794  0013  2815               	goto	u35_21
  1795  0014  2816               	goto	u35_20
  1796  0015                     u35_21:
  1797  0015  281B               	goto	i1l846
  1798  0016                     u35_20:
  1799  0016  2817               	goto	i1l842
  1800                           opt subtitle "HI-TECH Software Omniscient Code Generator (Lite mode) build 49521"
  1801  0017                     i1l102:	
  1802                           opt subtitle "HI-TECH Software Omniscient Code Generator (Lite mode) build 49521"
  1803                           
  1804  0017                     i1l842:	
  1805                           opt subtitle "HI-TECH Software Omniscient Code Generator (Lite mode) build 49521"
  1806  0017  019D               	clrf	(413)^0180h	;volatile
  1807                           opt subtitle "HI-TECH Software Omniscient Code Generator (Lite mode) build 49521"
  1808                           
  1809  0018                     i1l844:	
  1810                           opt subtitle "HI-TECH Software Omniscient Code Generator (Lite mode) build 49521"
  1811  0018  3090               	movlw	(090h)
  1812  0019  009D               	movwf	(413)^0180h	;volatile
  1813                           opt subtitle "HI-TECH Software Omniscient Code Generator (Lite mode) build 49521"
  1814                           
  1815  001A  2849               	goto	i1l106
  1816                           opt subtitle "HI-TECH Software Omniscient Code Generator (Lite mode) build 49521"
  1817                           
  1818  001B                     i1l100:	
  1819                           opt subtitle "HI-TECH Software Omniscient Code Generator (Lite mode) build 49521"
  1820                           
  1821  001B                     i1l846:	
  1822                           opt subtitle "HI-TECH Software Omniscient Code Generator (Lite mode) build 49521"
  1823                           
  1824  001B  0871               	movf	(_Index+1),w
  1825  001C  3A80               	xorlw	80h
  1826  001D  00FF               	movwf	btemp+1
  1827  001E  3081               	movlw	(high(0100h))^80h
  1828  001F  027F               	subwf	btemp+1,w
  1829  0020  1D03               	skipz
  1830  0021  2824               	goto	u36_25
  1831  0022  3000               	movlw	low(0100h)
  1832  0023  0270               	subwf	(_Index),w
  1833  0024                     u36_25:
  1834                           opt subtitle "HI-TECH Software Omniscient Code Generator (Lite mode) build 49521"
  1835  0024  1803               	skipnc
  1836  0025  2827               	goto	u36_21
  1837  0026  2828               	goto	u36_20
  1838  0027                     u36_21:
  1839  0027  2840               	goto	i1l852
  1840  0028                     u36_20:
  1841                           opt subtitle "HI-TECH Software Omniscient Code Generator (Lite mode) build 49521"
  1842                           
  1843  0028                     i1l848:	
  1844                           opt subtitle "HI-TECH Software Omniscient Code Generator (Lite mode) build 49521"
  1845  0028  0023               	movlb 3	; select bank3
  1846  0029  0819               	movf	(409)^0180h,w	;volatile
  1847  002A  00F6               	movwf	(??_isr+0)+0
  1848  002B  3070               	movlw	low(8304)
  1849  002C  00F7               	movwf	(??_isr+1)+0
  1850  002D  3020               	movlw	high(8304)
  1851  002E  00F8               	movwf	(??_isr+1)+0+1
  1852  002F  0870               	movf	(_Index),w
  1853  0030  0777               	addwf	0+(??_isr+1)+0,w
  1854  0031  00F9               	movwf	(??_isr+3)+0
  1855  0032  0871               	movf	(_Index+1),w
  1856  0033  3D78               	addwfc	1+(??_isr+1)+0,w
  1857  0034  00FA               	movwf	1+(??_isr+3)+0
  1858  0035  0879               	movf	0+(??_isr+3)+0,w
  1859  0036  0086               	movwf	fsr1l
  1860  0037  087A               	movf	1+(??_isr+3)+0,w
  1861  0038  0087               	movwf	fsr1h
  1862                           opt subtitle "HI-TECH Software Omniscient Code Generator (Lite mode) build 49521"
  1863  0039  0876               	movf	(??_isr+0)+0,w
  1864  003A  0081               	movwf	indf1
  1865                           opt subtitle "HI-TECH Software Omniscient Code Generator (Lite mode) build 49521"
  1866  003B                     i1l850:	
  1867  003B  3001               	movlw	low(01h)
  1868  003C  07F0               	addwf	(_Index),f
  1869  003D  3000               	movlw	high(01h)
  1870  003E  3DF1               	addwfc	(_Index+1),f
  1871                           opt subtitle "HI-TECH Software Omniscient Code Generator (Lite mode) build 49521"
  1872                           
  1873  003F  2849               	goto	i1l106
  1874                           opt subtitle "HI-TECH Software Omniscient Code Generator (Lite mode) build 49521"
  1875                           
  1876  0040                     i1l104:	
  1877                           opt subtitle "HI-TECH Software Omniscient Code Generator (Lite mode) build 49521"
  1878                           
  1879  0040                     i1l852:	
  1880                           opt subtitle "HI-TECH Software Omniscient Code Generator (Lite mode) build 49521"
  1881                           
  1882  0040  0023               	movlb 3	; select bank3
  1883  0041  0819               	movf	(409)^0180h,w	;volatile
  1884  0042  00F6               	movwf	(??_isr+0)+0
  1885  0043  0876               	movf	(??_isr+0)+0,w
  1886  0044  0020               	movlb 0	; select bank0
  1887  0045  00C5               	movwf	(_rcv)
  1888  0046  2849               	goto	i1l106
  1889                           opt subtitle "HI-TECH Software Omniscient Code Generator (Lite mode) build 49521"
  1890  0047                     i1l105:	
  1891  0047  2849               	goto	i1l106
  1892                           opt subtitle "HI-TECH Software Omniscient Code Generator (Lite mode) build 49521"
  1893                           
  1894  0048                     i1l103:	
  1895  0048  2849               	goto	i1l106
  1896                           opt subtitle "HI-TECH Software Omniscient Code Generator (Lite mode) build 49521"
  1897                           
  1898  0049                     i1l99:	
  1899                           opt subtitle "HI-TECH Software Omniscient Code Generator (Lite mode) build 49521"
  1900                           
  1901  0049                     i1l106:	
  1902  0049  087B               	movf	(??_isr+5),w
  1903  004A  0020               	movlb 0	; select bank0
  1904  004B  00FF               	movwf	btemp+1
  1905  004C  0009               	retfie
  1906                           opt subtitle "HI-TECH Software Omniscient Code Generator (Lite mode) build 49521"
  1907                           
  1908  004D                     	__end_of_isr:
  1909                           opt subtitle "HI-TECH Software Omniscient Code Generator (Lite mode) build 49521"
  1910                           
  1911                           opt pagewidth 120
  1912  007E                     	btemp set 07Eh
  1913                           opt subtitle "HI-TECH Software Omniscient Code Generator (Lite mode) build 49521"
  1914                           
  1915                           opt pagewidth 120
  1916  007E                     	wtemp0 set btemp
  1917                           opt subtitle "HI-TECH Software Omniscient Code Generator (Lite mode) build 49521"
  1918  2070                     __pbssBIGRAM	equ	8304


Data Sizes:
    Strings     0
    Constant    0
    Data        29
    BSS         7
    Persistent  0
    Stack       0

Auto Spaces:
    Space          Size  Autos    Used
    COMMON           14      6      12
    BANK0            80      8      38
    BANK1            32      0       0
    BANK2             0      0       0
    BANK3             0      0       0
    BANK4             0      0       0

Pointer List with Targets:

    None.

Critical Paths under _main in COMMON

    None.

Critical Paths under _isr in COMMON

    None.

Critical Paths under _main in BANK0

    _main->_Delayms

Critical Paths under _isr in BANK0

    None.

Critical Paths under _main in BANK1

    None.

Critical Paths under _isr in BANK1

    None.

Critical Paths under _main in BANK2

    None.

Critical Paths under _isr in BANK2

    None.

Critical Paths under _main in BANK3

    None.

Critical Paths under _isr in BANK3

    None.

Critical Paths under _main in BANK4

    None.

Critical Paths under _isr in BANK4

    None.

Call Graph Tables:

 ---------------------------------------------------------------------------------
 (Depth) Function   	        Calls       Base Space   Used Autos Params    Refs
 ---------------------------------------------------------------------------------
 (0) _main                                                 6     6      0      62
                                              2 BANK0      6     6      0
                            _Delayms
                               _Send
 ---------------------------------------------------------------------------------
 (1) _Delayms                                              2     0      2      31
                                              0 BANK0      2     0      2
 ---------------------------------------------------------------------------------
 (1) _Send                                                 1     1      0      31
                                              0 BANK0      1     1      0
 ---------------------------------------------------------------------------------
 Estimated maximum stack depth 1
 ---------------------------------------------------------------------------------
 (Depth) Function   	        Calls       Base Space   Used Autos Params    Refs
 ---------------------------------------------------------------------------------
 (2) _isr                                                  6     6      0       0
                                              0 COMMON     6     6      0
 ---------------------------------------------------------------------------------
 Estimated maximum stack depth 2
 ---------------------------------------------------------------------------------

 Call Graph Graphs:

 _main (ROOT)
   _Delayms
   _Send

 _isr (ROOT)

 Address spaces:
Name               Size   Autos  Total    Cost      Usage
BIGRAM             170      0       0       0        0.0%
EEDATA             100      0       0       0        0.0%
NULL                 0      0       0       0        0.0%
CODE                 0      0       0       0        0.0%
BITCOMMON            E      0       0       1        0.0%
BITSFR0              0      0       0       1        0.0%
SFR0                 0      0       0       1        0.0%
COMMON               E      6       C       2       85.7%
BITSFR1              0      0       0       2        0.0%
SFR1                 0      0       0       2        0.0%
BITSFR2              0      0       0       3        0.0%
SFR2                 0      0       0       3        0.0%
STACK                0      0       1       3        0.0%
BITSFR3              0      0       0       4        0.0%
SFR3                 0      0       0       4        0.0%
ABS                  0      0      32       4        0.0%
BITBANK0            50      0       0       5        0.0%
BITSFR4              0      0       0       5        0.0%
SFR4                 0      0       0       5        0.0%
BANK0               50      8      26       6       47.5%
BITSFR5              0      0       0       6        0.0%
SFR5                 0      0       0       6        0.0%
BITBANK1            50      0       0       7        0.0%
BITSFR6              0      0       0       7        0.0%
SFR6                 0      0       0       7        0.0%
BANK1               20      0       0       8        0.0%
BITSFR7              0      0       0       8        0.0%
SFR7                 0      0       0       8        0.0%
BITBANK2            50      0       0       9        0.0%
BITSFR8              0      0       0       9        0.0%
SFR8                 0      0       0       9        0.0%
BITSFR9              0      0       0      10        0.0%
SFR9                 0      0       0      10        0.0%
BANK2                0      0       0      10        0.0%
BITBANK3            50      0       0      11        0.0%
BITSFR10             0      0       0      11        0.0%
SFR10                0      0       0      11        0.0%
BITSFR11             0      0       0      12        0.0%
SFR11                0      0       0      12        0.0%
BANK3                0      0       0      12        0.0%
BITBANK4            30      0       0      13        0.0%
BITSFR12             0      0       0      13        0.0%
SFR12                0      0       0      13        0.0%
BITSFR13             0      0       0      14        0.0%
SFR13                0      0       0      14        0.0%
BANK4                0      0       0      14        0.0%
BITSFR14             0      0       0      15        0.0%
SFR14                0      0       0      15        0.0%
DATA                 0      0      33      15        0.0%
BITSFR15             0      0       0      16        0.0%
SFR15                0      0       0      16        0.0%
BITSFR16             0      0       0      17        0.0%
SFR16                0      0       0      17        0.0%
BITSFR17             0      0       0      18        0.0%
SFR17                0      0       0      18        0.0%
BITSFR18             0      0       0      19        0.0%
SFR18                0      0       0      19        0.0%
BITSFR19             0      0       0      20        0.0%
SFR19                0      0       0      20        0.0%
BITSFR20             0      0       0      21        0.0%
SFR20                0      0       0      21        0.0%
BITSFR21             0      0       0      22        0.0%
SFR21                0      0       0      22        0.0%
BITSFR22             0      0       0      23        0.0%
SFR22                0      0       0      23        0.0%
BITSFR23             0      0       0      24        0.0%
SFR23                0      0       0      24        0.0%
BITSFR24             0      0       0      25        0.0%
SFR24                0      0       0      25        0.0%
BITSFR25             0      0       0      26        0.0%
SFR25                0      0       0      26        0.0%
BITSFR26             0      0       0      27        0.0%
SFR26                0      0       0      27        0.0%
BITSFR27             0      0       0      28        0.0%
SFR27                0      0       0      28        0.0%
BITSFR28             0      0       0      29        0.0%
SFR28                0      0       0      29        0.0%
BITSFR29             0      0       0      30        0.0%
SFR29                0      0       0      30        0.0%
BITSFR30             0      0       0      31        0.0%
SFR30                0      0       0      31        0.0%
BITSFR31             0      0       0      32        0.0%
SFR31                0      0       0      32        0.0%


Microchip Technology PIC Macro Assembler V1.12 build 49521 
Symbol Table                                                                                   Sat Dec 29 09:51:30 2012

                      _i 0072              __CFG_CP$OFF 0000                       l70 0092  
                     l71 00EB                       l80 00E0                       l72 0093  
                     l81 00E1                       l73 0094                       l90 018A  
                     l82 00E3                       l74 00A9                       l91 0177  
                     l83 00E5                       l75 00B9                       l67 0082  
                     l92 016A                       l68 0130                       l76 011C  
                     l84 00E7                       l93 0181                       l69 011D  
                     l85 00E9                       l77 00BA                       l94 018B  
                     l86 012D                       l78 00BB                       l95 018C  
                     l87 0162                       l79 00D0                       l96 018C  
                     l88 014A                       l89 015A                      l110 01EF  
                    l111 01F5                      l112 01F9                      l120 01CE  
                    l121 01CE                      l115 01BF                      l116 01B8  
                    l109 01EF                      l117 01B9                      l118 01B9  
                    l119 01BD                      l900 009C                      l910 00B2  
                    l902 00A1                      l920 00D0                      l912 00BB  
                    l904 00A8                      l922 00D4                      l914 00C3  
                    l906 00A9                      l930 011D                      l940 0142  
                    l932 012D                      l924 00D9                      l916 00C8  
                    l908 00AD                      l860 0059                      l942 0149  
                    l950 015A                      l926 00EA                      l918 00CF  
                    l934 0130                      l870 0067                      l862 005B  
                    l854 004F                      l960 0177                      l944 014A  
                    l936 0135                      l952 0162                      l928 00EB  
                    l880 0073                      l872 006A                      l864 005D  
                    l856 0055                      l970 01EE                      l962 0181  
                    l954 0167                      l946 014E                      l938 013D  
                    l890 007F                      l882 0075                      l874 006C  
                    l866 005E                      l858 0056                      l972 01F5  
                    l964 01B1                      l956 016A                      l948 0153  
                    l892 0080                      l884 0077                      l876 006F  
                    l868 0065                      l966 01B3                      l958 0172  
                    l894 0082                      l886 007C                      l878 0071  
                    l968 01BF                      l896 008F                      l888 007D  
                    l898 0094                      _RB3 006B                      _RB4 006C  
                    u400 00CE                      u401 00CD                      u410 00DF  
                    u411 00DE                      u500 01F4                      u420 012C  
                    u501 01F3                      u421 012B                      u430 0135  
                    _PR2 001B                      u431 0134                      u440 0148  
                    u441 0147                      u425 0128                      u450 0159  
                    u370 008F             __CFG_CPD$OFF 0000                      u451 0158  
                    u371 008E                      u460 0167                      u380 00A7  
                    u461 0166                      u381 00A6                      u470 0180  
                    u390 00B8                      u471 017F                      u391 00B7  
                    u375 008B                      u480 01BD                      u481 01BC  
                    u490 01CD                      u491 01CC                      u495 01C9  
                    _Buf 2070                      _Msg 0020                      _isr 0004  
                    _rcv 0045             __CFG_BORV$LO 0000             __CFG_LVP$OFF 0000  
                   ?_isr 0076                     i1l99 0049                     _WPUB 020D  
           __CFG_WRT$OFF 0000                     _Send 01EC                     _data 0075  
                   _main 004F                     fsr0h 0005                     fsr1h 0007  
                   fsr0l 0004                     indf0 0000                     indf1 0001  
                   fsr1l 0006                     btemp 007E            __CFG_BOREN$ON 0000  
                   start 004D            __CFG_IESO$OFF 0000          __end_of_Delayms 01CF  
          __CFG_MCLRE$ON 0000                    ??_isr 0076            __CFG_PLLEN$ON 0000  
                  ?_Send 0076                    ?_main 0076            __CFG_WDTE$OFF 0000  
                  _T2CON 001C                    i1l100 001B                    i1l102 0017  
                  i1l103 0048                    i1l104 0040                    i1l105 0047  
                  i1l106 0049                    i1l840 0012                    i1l850 003B  
                  i1l842 0017                    i1l852 0040                    i1l844 0018  
                  i1l836 0008                    i1l846 001B                    i1l838 000C  
                  i1l848 0028                    _RCREG 0199                    _RCSTA 019D  
                  u33_20 000C                    u33_21 000B                    u34_20 0012  
                  u34_21 0011                    _SPBRG 019B                    u35_20 0016  
                  u35_21 0015                    u36_20 0028                    u36_21 0027  
                  u36_25 0024                    _TRISA 008C                    _TRISB 008D  
                  _TXREG 019A                    _TXSTA 019E            __CFG_PWRTE$ON 0000  
                  _Index 0070           __CFG_FCMEN$OFF 0000                    _ascii 0074  
                  wtemp0 007E          __initialization 018E             __end_of_Send 01FA  
           __end_of_main 018E                   ??_Send 003D                   ??_main 003F  
                 _ANSELA 018C                   _ANSELB 018D                ??_Delayms 003F  
                 _OSCCON 0099                   clrloop 01FB  __end_of__initialization 01AE  
         __pcstackCOMMON 0076             __pidataBANK0 01CF           _OPTION_REGbits 0095  
             __pbssBANK0 0045               __pmaintext 004F               __pintentry 0004  
                _BAUDCON 019F                  _Delayms 01B1          __CFG_STVREN$OFF 0000  
           __size_of_isr 0049     end_of_initialization 01AE                  init_ram 0206  
                initloop 0207         __CFG_CLKOUTEN$ON 0000                _RCSTAbits 019D  
              _PORTAbits 000C         __CFG_FOSC$INTOSC 0000                _TXSTAbits 019E  
    start_initialization 018E              __end_of_isr 004D              __pdataBANK0 0020  
            __pbssBIGRAM 2070              __pbssCOMMON 0070            __pcstackBANK0 003D  
               ?_Delayms 003D                __ptext143 01B1                __ptext144 01EC  
               _PIE1bits 0091                 Delayms@t 003D                 _PIR1bits 0011  
               Send@Data 003D         __size_of_Delayms 001E            __size_of_Send 000E  
          __size_of_main 013F                 clear_ram 01FA               _INTCONbits 000B  
               intlevel1 0000  
